:020000040800F2
:1000000000AF002001020008412D00086918000817
:10001000352C0008090D00085936000800000000C2
:10002000000000000000000000000000490100087E
:100030009D0D0008000000009D010008E934000843
:100040001B0200081B0200081B0200081B0200081C
:100050001B0200081B0200081B0200081B0200080C
:100060001B0200081B0200081B0200081B020008FC
:100070001B0200081B0200081B0200081B020008EC
:100080001B0200081B0200081B0200081B020008DC
:100090001B0200081B0200081B0200081B020008CC
:1000A0001B0200081B0200081B0200081B020008BC
:1000B000813500081B0200081B0200081B02000813
:1000C0001B0200081B0200081B0200081B0200089C
:1000D0001B02000895350008053600081B020008C1
:1000E0001B0200081B0200081B0200081B0200087C
:1000F0001B0200081B0200081B0200081B0200086C
:100100001B0200081B0200081B0200081B0200085B
:100110001B0200081B0200081B0200081B0200084B
:100120001B0200081B0200081B0200081B0200083B
:10013000DFF810D000F0F0FA0048004735730008EF
:10014000AFF3008000AF00202A4B19680868B0E8C0
:10015000F04F80F30988BFF36F8F4FF0000080F3FA
:10016000118870470000000006480068006880F3AE
:10017000088862B661B6BFF34F8FBFF36F8F00DFA1
:1001800000BF00BF08ED00E0DFF80C00016841F49B
:1001900070010160704700BF88ED00E0EFF3098057
:1001A000BFF36F8F134B1A681EF0100F08BF20EDBE
:1001B000108A20E9F04F106008B44FF0500080F32F
:1001C0001188BFF34F8FBFF36F8F09F0B5FF4FF06A
:1001D000000080F3118808BC19680868B0E8F04F87
:1001E0001EF0100F08BFB0EC108A80F30988BFF32F
:1001F0006F8F7047F0000020EFF30580704700001C
:100200000648804706480047FEE7FEE7FEE7FEE7B0
:10021000FEE7FEE7FEE7FEE7FEE7FEE7FD34000847
:100220003101000840EA01039B0703D009E008C937
:10023000121F08C0042AFAD203E011F8013B00F8AB
:10024000013B521EF9D27047D2B201E000F8012BF7
:10025000491EFBD270470022F6E710B513460A4646
:1002600004461946FFF7F0FF204610BD30B504469E
:100270000020034600E05B1C934203D2E05CCD5CAF
:10028000401BF8D030BD2DE9FE4F804681EA0300C7
:10029000C00F0C46009021F0004123F00045B8EB60
:1002A0000200A94105D24046214690461C460B4615
:1002B000024623F00040104347D0270DC7F30A0041
:1002C000C3F30A510290401A019040286BDAC3F33D
:1002D000130040F4801B0098924620B10023D2EB1B
:1002E000030A63EB0B0B01985946C0F140025046DC
:1002F00000F04DF906460D4650465946019A00F069
:1003000065F910EB08006141002487EA115284EA84
:10031000E7731A4340D0009A62B3019A012A4FEA68
:10032000075215DC001B61EB02014FF0004202EAAC
:100330000752CDE90042001C41F5801132462B46A0
:1003400000F09CF903B0BDE8F08F40462146F9E784
:10035000001B61EB0201001C41F5801300185B419A
:100360002018A2F5001747EB030140EAD570B61933
:100370006D4111E06D084FEA360645EAC0754FEA57
:100380000752001B61EB0201001C41F58011490876
:100390004FEA30000019514132462B4603B0BDE808
:1003A000F04F00F05CB90098012240000023D0EB30
:1003B000020263EBE073009821464FEAE074B8EB69
:1003C000000061EB0401E9E783F000435BE781F0A3
:1003D000004158E72DE9FE4F81EA030404F0004490
:1003E00021F0004100944FF0000B23F0004350EA4D
:1003F00001045ED052EA03045BD0C3F30A54C1F394
:100400000A552C44A4F2F3340194A0FB0254C1F326
:10041000130141F48011C3F3130343F4801301FB70
:10042000024400FB034E840A970A44EA815447EAD7
:100430008357A4FB076802958D0A05FB07854FEAE1
:10044000932C04FB0C542705029D4FEA065847EAFB
:100450001637B5EB08056EEB070C870E920E47EAD0
:10046000811742EA8312A7FB0201B6EB0B0164EB92
:1004700000042B0D43EA0C335E1844EB1C50DA46A3
:100480005146E7FB0201C5F313044FEA0B3343EA7D
:1004900014534FEA0432019C43EA0603A4F10C040E
:1004A0000294009CCDE900B400F0E8F803B0BDE888
:1004B000F08F00200146F9E70EB540F2334102917A
:1004C0000021CDE900110A460B4600F0D7F803B031
:1004D00000BDC1F30A5210B5C1F3130140F2FF335E
:1004E00041F480119A4201DA002010BD40F23343FA
:1004F0009A42A2F2334203DC524200F057F810BD98
:10050000904010BD00F0004230F000400AD0C10D14
:1005100001F56071C0F3160042EA0151C2084007BC
:100520001143704700200146704701F0004330B48A
:1005300021F0004150EA010206D00A0DA2F56072D6
:10054000C1F31301002A02DC30BC00207047440FC5
:1005500044EAC104C100E01830BC00EBC25000F016
:1005600047B830B50B46014600202022012409E09F
:1005700021FA02F59D4205D303FA02F5491B04FA5C
:1005800002F52844151EA2F10102F1DC30BD202A3B
:1005900004DB203A00FA02F1002070479140C2F1DA
:1005A000200320FA03F3194390407047202A04DB0C
:1005B000203A21FA02F00021704721FA02F3D040DC
:1005C000C2F120029140084319467047202A06DBF9
:1005D000CB17203A41FA02F043EAE07306E041FA11
:1005E00002F3D040C2F120029140084319467047FF
:1005F0000029A8BF7047401C490008BF20F0010037
:10060000704710B4B0FA80FC00FA0CF050EA010414
:1006100004BF10BC704749B1CCF1200421FA04F4A6
:1006200011FA0CF118BF012121430843A3EB0C017F
:10063000CB1D4FEA00614FEA102042BF002010BCE2
:10064000704700EBC35010440029A4BF10BC704792
:10065000401C490008BF20F0010010BC704710B5D5
:10066000141E73F1000408DA401C41F100019218D5
:100670005B411A4301D120F0010010BD2DE9F04D7E
:1006800092469B4611B1B1FA81F202E0B0FA80F2D3
:1006900020329046FFF77BFF04460F4640EA0A00EF
:1006A00041EA0B0153465A46084313D0114653EA18
:1006B000010019D0C8F140025046FFF777FF054608
:1006C0000E46504659464246FFF761FF084305D0A3
:1006D000012004E020463946BDE8F08D00200543A6
:1006E00046EAE0762C4337430A986305E40AA0EB18
:1006F00008000022FD0A44EA47540A3002D50020CF
:100700000146E9E7010510196941DDE908450019CD
:100710006941BDE8F04DA2E7064C074D06E0E068F0
:1007200040F0010394E8070098471034AC42F6D338
:10073000FFF702FD6CB300088CB3000830B58C18CD
:1007400010F8012B12F00F0301D110F8013B120930
:1007500006D110F8012B03E010F8015B01F8015BF2
:100760005B1EF9D101E001F8013B521EFBD1A14211
:10077000E6D3002030BD0000044890F84200400756
:1007800001D40120704700207047000098AA002083
:10079000044890F84200C00701D0002070470120B3
:1007A0007047000098AA002000B5A3B00C49088D3E
:1007B000012812D0002001908DF8040088788DF86F
:1007C000050002AA01A9012002F066FA05480023EB
:1007D0001A4602A9006809F013FF23B000BD00000B
:1007E00098AA00202400002000B5A3B00D49088D70
:1007F000012814D0002001908DF80400087800F042
:100800000F008DF8050002AA01A9022002F044FAA7
:10081000054800231A4602A9006809F0F1FE23B03A
:1008200000BD000098AA002024000020F0B5A3B06D
:10083000304E308D012833D0F08E2F4F002560B11F
:1008400001282DD101240195012C2BD0022C2FD071
:10085000032C33D0042C3DD137E0009501958DF861
:100860000050B0788DF801008DF8025030788DF886
:100870000300F088010A8DF804108DF805008DF84A
:10088000065030798DF8070002AB6A46042101203A
:1008900002F024FA00231A4602A9386809F0B0FED3
:1008A00023B0F0BD8DF80450B0788DF8050011E04C
:1008B0008DF8045030788DF805000BE0F088010ABF
:1008C0008DF804108DF8050004E08DF8045030799F
:1008D0008DF8050002AA01A9204602F0DDF90023E7
:1008E0001A4602A9386809F08BFE641CE4B2052C94
:1008F000A9D3D5E798AA0020240000202DE9F05FB5
:100900000546DDE90A9B884614461E46B9F1000FEC
:1009100055D05349534800270A8803889A4207D084
:100920002F7088F8007004B1277037707770B77037
:10093000DFF82CA1BAF800100180BAF804004FF6D5
:10094000FF7100EB800001EA400002F0F7FC024674
:10095000BAF800004FF0010A70B14149012837D0C0
:10096000884602285BD0032829D1B8F80600314612
:10097000BDE8F05F02F071BEB9F1020F05D15FEA88
:100980008B7001D5012200E00422501E022804D8F9
:1009900085F800A044B1277006E0101F022803D894
:1009A0002F700CB184F800A02878012809D02C49B8
:1009B000B1F84A10012904D0002800D13770BDE8F1
:1009C000F09F27483146C088BDE8F05F02F045BE81
:1009D000B9F1020F05D15FEA8B6001D5042200E076
:1009E0000122101F022804D888F800A04CB12770FB
:1009F00007E0501E022804D888F800700CB184F873
:100A000000A098F80000012803D00028D7D1377043
:100A1000D5E7C8883146BDE8F05F02F01EBEE6208B
:100A200002F08CFC0246501E022804D885F800A073
:100A300044B1277006E0101F022803D82F700CB1B4
:100A400084F800A02878012803D00028B7D1377097
:100A5000B5E7B8F806003146BDE8F05F02F0FDBD2D
:100A600098AA0020AA01002000B5A3B00C49088D67
:100A7000012812D0002001908DF8040008798DF82B
:100A8000050002AA01A9042002F006F90548002386
:100A90001A4602A9006809F0B3FD23B000BD0000AA
:100AA00098AA00202400002000B5A3B01C4A108D95
:100AB000012832D000201B49CB78012B06D00B79BE
:100AC000012B05D04979012904D004E0012002E07E
:100AD000012000E00120D288130A02F00F0101EB8F
:100AE0000011C9B2D20506D510B1012802D002E02A
:100AF000002100E01021002001908DF804308DF8D5
:100B0000051002AA01A9032002F0C6F80648002336
:100B10001A4602A9006809F073FD23B000BD000069
:100B200098AA00207700002024000020704710B50C
:100B300008F048F908F0A0F908F038FABDE81040CC
:100B400008F086BA7FB504464FF4E06007F0ACFDCC
:100B5000684608F060FD4FF08045284608F086FCA6
:100B60007720ADF800000021ADF80210ADF80410B8
:100B70000294ADF806106946284608F0EFFC2846B6
:100B800008F01CFB002206211C2006F035FE012186
:100B9000284608F031FD0121284608F029FD2846A5
:100BA00008F0D7FC7FBD000070B505464FF4A0608B
:100BB00006F070FE00221146262006F01DFE40F2CF
:100BC000026007F071FD40F2046007F06DFD40F235
:100BD000117007F069FD4FF48043032210211F4874
:100BE00005F04CFF1E4C082303220421204605F08B
:100BF00045FF042303221821204605F03FFF194C2E
:100C0000204608F0ABFD2946204608F02FFD0021C4
:100C1000204608F06BFE0021204608F055FE00211A
:100C2000204608F03FFE0021204608F0FBFD002191
:100C3000204608F0EDFD0421204608F03BFE082187
:100C4000204608F049FE204608F0D0FD2046BDE8C9
:100C5000704040F2053108F0F9BD0000001001407D
:100C6000000801400044004010B505F095FF08F071
:100C700035FD01F0BFFE03F04FF9FFF758FF0548BF
:100C8000408E00F009F802F0C1F9BDE810400AF00A
:100C900087B9000098AA002070B54FF41655B0F53A
:100CA000F07F20D0B0F5707F20D0B0F5B46F1FD0AA
:100CB000B0F5F06F1FD0B0F5706F1FD0B0F5AF5F1B
:100CC0001FD14DF6C0242046FFF76EFFAC4200D97D
:100CD0002C460C48B0FBF4F080B2FFF733FFBDE8C0
:100CE000704005F02DBB4FF49654ECE72C46EAE734
:100CF0004FF46154E7E74FF49644E4E74FF41644A9
:100D0000E1E770BD80F0FA02FEE730B505460C461B
:100D1000A01EC1B2284600F061FC82B2110AD2B214
:100D2000281910F8023C8B4205D110F8010C9042B2
:100D300001D1012030BD002030BD000010B5094CAC
:100D4000012060704FF47A7008F0E2FF0648408E90
:100D5000FFF7A2FF002060706068BDE8104009F056
:100D600069B800009401002098AA002070B50446DC
:100D7000054D06A0298802F045FD2888002802D0EC
:100D80002078401C207070BDD8AA00205061726D80
:100D90005F536176652025640D0A00007047704737
:100DA0007047704770B500EE100AB2EE041AF8EE04
:100DB000400A80EE810A10EE100AFFF7A3FB9FEDB8
:100DC000191B53EC112BFFF75EFAFFF782FB80B281
:100DD00000EB80004FF6FF7101EA40004FF47A719A
:100DE000B0FBF1F201FB12016422B1FBF2F1C9B2D6
:100DF000B0FBF2F302FB13030A22B3FBF2F5B0FBE4
:100E0000F2F302FB130411B1012000F03FF8294670
:100E1000022000F03BF82146BDE87040032000F0BE
:100E200035B80000000000000000E03F70B5002869
:100E300000DA404200B24FF47A7190FBF1F201FB0C
:100E40001201642291FBF2F1C9B290FBF2F302FBB2
:100E500013030A2293FBF2F3DCB290FBF2F302FBE2
:100E60001300C5B261B1012000F010F82146022044
:100E700000F00CF82946BDE87040032000F006B8E9
:100E800008210120FFF78CFFF0E7000030B4F74A9B
:100E9000012804D0022875D0032874D087E2F348D3
:100EA0000A29038843F4006023F40063F6D2DFE8E4
:100EB00001F005192D41556B7F93A7BBD18841F0F7
:100EC000040141F40061D180918821F0040141F4D2
:100ED00000619180518841F0040141F4006151802A
:100EE000108064E2D08820F0040020F40060D080FC
:100EF000908820F0040040F400609080508820F03A
:100F0000040040F400605080138050E2D18821F04A
:100F1000040141F40061D180918841F0040141F461
:100F200000619180518841F0040121F400615180F9
:100F300010803CE2D18821F0040141F40061D180AD
:100F4000918841F0040141F400619180518821F0C1
:100F5000040141F400615180108028E2D08840F003
:100F6000040020F40060D080908840F0040040F439
:100F700000609080508820F0040040F400605080B1
:100F8000138014E264E03AE1D18841F0040141F4B5
:100F90000061D180918841F0040121F400619180C9
:100FA000518821F0040141F4006151801080FEE17C
:100FB000D18841F0040141F40061D180918841F071
:100FC000040121F400619180518841F0040141F451
:100FD000006151801080EAE1D08820F0040040F4E4
:100FE0000060D080908820F0040040F40060908081
:100FF000508820F0040040F4006050801380D6E157
:10100000D18841F0040141F40061D180918841F020
:10101000040141F400619180518841F0040141F4E0
:10102000006151801080C2E1D18841F0040141F497
:101030000061D180918841F0040141F40061918008
:10104000518821F0040141F4006151801080AEE12B
:1010500086480A29038843F4007023F4007390D271
:10106000DFE801F005192D4155697D91A5B9D188B9
:1010700041F4806141F40071D180918821F4806154
:1010800041F400719180518841F4806141F4007114
:10109000518010808BE1D08820F4806020F40070B3
:1010A000D080908820F4806040F400709080508858
:1010B00020F4806040F400705080138077E1D18884
:1010C00021F4806141F40071D180918841F4806104
:1010D00041F400719180518841F4806121F40071E4
:1010E0005180108063E1D18821F4806141F4007166
:1010F000D180918841F4806141F4007191805188E0
:1011000021F4806141F40071518010804FE1D0885A
:1011100040F4806020F40070D080908840F48060BB
:1011200040F400709080508820F4806040F400709B
:10113000508013803BE1D18841F4806141F400711B
:10114000D180918841F4806121F4007191805188AF
:1011500021F4806141F400715180108027E1D18831
:1011600041F4806141F40071D180918841F4806143
:1011700021F400719180518841F4806141F4007143
:101180005180108013E1D08820F4806040F400701A
:10119000D080908820F4806040F400709080508867
:1011A00020F4806040F4007050801380FFE0D1880C
:1011B00041F4806141F40071D180918841F48061F3
:1011C00041F400719180518841F4806141F40071D3
:1011D00051801080EBE0D18841F4806141F40071CE
:1011E000D180918841F4806141F4007191805188EF
:1011F00021F4806141F4007151801080D7E01B48D8
:101200000A29038843F0400023F0400319D2DFE8A5
:1012100001F005192F43576B7F93A7BBD18841F08D
:10122000800141F04001D180918821F0800141F09E
:1012300040019180518841F0800141F0400151808E
:101240001080B4E0D08820F0800020F04000D080F2
:10125000908820F0800040F040009080508820F07E
:10126000800040F0400050801380A0E05C0000202F
:10127000D18821F0800141F04001D180918841F076
:10128000800141F040019180518841F0800121F0BE
:101290004001518010808AE0D18821F0800141F026
:1012A0004001D180918841F0800141F0400191805E
:1012B000518821F0800141F040015180108076E09A
:1012C000D08840F0800020F04000D080908840F02E
:1012D000800040F040009080508820F0800040F076
:1012E00040005080138062E0D18841F0800141F0DD
:1012F0004001D180918841F0800121F0400191802E
:10130000518821F0800141F04001518010804EE071
:10131000D18841F0800141F04001D180918841F0B5
:10132000800121F040019180518841F0800141F01D
:101330004001518010803AE0D08820F0800040F0D9
:101340004000D080908820F0800040F040009080E5
:10135000508820F0800040F040005080138026E04C
:10136000D18841F0800141F04001D180918841F065
:10137000800141F040019180518841F0800141F0AD
:1013800040015180108012E0D18841F0800141F08D
:101390004001D180918841F0800141F0400191806D
:1013A000518821F0800141F040015180108030BC13
:1013B00000F0BABF10B5164C00290FD0012926D174
:1013C000002818DBFFF732FD2088012140F0800261
:1013D0002280BDE81040072005F00EBC80B2FFF768
:1013E000E1FC2088012140F080022280BDE810400D
:1013F000072005F001BCFFF7D4FC2088012120F074
:1014000080022280BDE81040072005F0F5BB10BD2A
:101410005C000020044890F84200800701D40120BD
:10142000704700207047000098AA0020F0B5174EC2
:101430004FF6FF77348F04EB840407EA4404F58900
:1014400005EB850507EA4505768F022A0BD1222B8D
:1014500002D0112B04D006E03219521C95B202E0E2
:101460002A19521C96B2371900220123AF4204D226
:101470000370002900D00A70F0BD2C44B442FBD2A6
:1014800002700029F8D00B70F0BD000098AA00206F
:1014900000B5A3B00C49088D012812D0002001909E
:1014A0008DF80400087B8DF8050002AA01A906202A
:1014B00001F0F2FB054800231A4602A9006809F072
:1014C0009FF823B000BD000098AA0020240000204F
:1014D00000B5A3B00C49088D012812D0002001905E
:1014E0008DF80400887B8DF8050002AA01A9072069
:1014F00001F0D2FB054800231A4602A9006809F052
:101500007FF823B000BD000098AA0020240000202E
:1015100000B5A3B00C49088D012812D0002001901D
:101520008DF80400087D8DF8050002AA01A90920A4
:1015300001F0B2FB054800231A4602A9006809F031
:101540005FF823B000BD000098AA0020240000200E
:10155000014602480022C08A02F07FB898AA002003
:1015600000B5A3B00C49088D012812D000200190CD
:101570008DF80400887D8DF8050002AA01A90B20D2
:1015800001F08AFB054800231A4602A9006809F009
:1015900037F823B000BD000098AA002024000020E6
:1015A00000B5A3B00B4A128D012A11D0002201927E
:1015B0008DF804008DF8051002AA01A90B2001F096
:1015C0006BFB054800231A4602A9006809F018F8C9
:1015D00023B000BD98AA00202400002070B5FF228F
:1015E000FF23084D05F5807605E010F8014B5440C7
:1015F0002A5D5A40335D491EC9B2F6D243EA022041
:1016000070BD00004CB10008F0B4034600204FF458
:1016100080611B4A1B4C4D01082B2ED2DFE803F0E2
:1016200004080E14191D2227F0BC104605F078BAE4
:10163000F0BC4FF48041104605F072BAF0BC4FF494
:101640008051104605F06CBA2046F0BC202105F010
:1016500067BAF0BC0C4805F063BA2946F0BC1046E6
:1016600005F05EBA29462046F0BC05F059BAF0BC38
:101670004FF40051104605F053BAF0BC704700001B
:10168000000C014000080140001001402DED0A8BC4
:101690000024002601F038FEDFF890A1DFF89091D9
:1016A0009FED649B654DDFF898816FF0080B9FED0F
:1016B00065AB9FED66BBB2EE04CA641C04215046C4
:1016C00005F035FA07460221624805F030FA074472
:1016D0000821504605F02BFA07440121504605F039
:1016E00026FA07440221504605F021FA3844C0B2D8
:1016F00010B19FED590B01E09FED590B51EC100B10
:10170000FEF713FF00EE100AA01B322834DD264638
:10171000D5ED080AF4EEC00AF1EE10FA16DB30EE51
:10172000C01A11EE100A484508DD10EE900AFEF7C7
:10173000E9FE53EC192BFEF747FE03E010EE100A0A
:10174000FEF7E0FEFEF7F1FE286215E030EE601ACB
:1017500011EE100A484508DD10EE900AFEF7D2FEA1
:1017600053EC192BFEF78FFD03E010EE100AFEF785
:10177000C9FEFEF7DAFE286298F92070092F01DD14
:10178000092703E05846874200DA074601F0BAFD10
:10179000F0EE40CAA869FEF7B5FE53EC1A2BFEF72F
:1017A00019FE00EE907A41EC180BB8EEE00AD5ED88
:1017B000080A3CEE800A30EE200A10EE100AFEF70E
:1017C000A1FE53EC1B2BFEF705FE53EC182BFEF786
:1017D0005AFDFEF7AAFE00EE100A85ED060A20EE7D
:1017E0000C0ABDEEC00A10EE100A00B2A8F83A00CA
:1017F0000A2190FBF1F1182005F086FE01F0EEFCC5
:10180000BCEEC00A10EE100AC0B200EE100AB8EE2C
:10181000400A85ED070ABCEEC00A10EE100AC0B2FD
:10182000A8F83C00C82008F073FA46E70010014011
:101830008FC2F53CB81E85EB51B89E3F6401002075
:1018400098AA0020CDCCCCCCCCCCEC3F9A999999DD
:101850009999B93F0008014000000000000012C043
:1018600000000000000004C0FEE7000010B540F2D8
:10187000036006F019FF094C4FF440630322102166
:10188000204605F0FBF8E114204605F0EFF821159D
:101890002046BDE8104005F0E9B80000000C01400A
:1018A00070B540F2026006F0FFFE40F2036006F001
:1018B000FBFE4FF4C06006F0F7FE01210F4805F073
:1018C0003DF901210E4805F039F90E4C1C23032285
:1018D0001021204605F0D2F80B4D012303221021E0
:1018E000284605F0CBF81C21204605F0BFF8284615
:1018F000BDE870400122114605F0BAB80001300081
:1019000000023000000C01400008014070B5104E8C
:101910004FF480652946304605F0A6F86C00234652
:1019200003221021304605F0A9F82146304605F083
:101930009DF800F0ADF82946304605F097F800F024
:10194000A7F829463046BDE8704005F08DB8000084
:10195000000C01402DE9F04780460024174E4FF45B
:1019600000694B4603224821304605F087F80025E0
:1019700037153946304605F077F800F089F83946D2
:10198000304605F073F86006040E4946304605F00F
:10199000C7F808B1641CE4B200F07AF86D1CEDB22F
:1019A000082DE6D3B8F1000F04D005F061F9204608
:1019B000BDE8F087FFF7AAFFF9E70000000C01403F
:1019C0002DE9F0410546184E4FF4006843460322C6
:1019D0001021304605F052F837153946304605F0EB
:1019E00043F80024280604D54146304605F03EF869
:1019F00003E04146304605F037F86806050E00F072
:101A000047F83946304605F031F800F041F83946DC
:101A1000304605F029F800F03BF8641CE4B2082CCD
:101A2000E0D3BDE8F0810000000C01402DE9F04159
:101A30000024164E4FF400652B4603224821304601
:101A400005F01CF82946304605F010F800F020F8A3
:101A50006F103946304605F009F800F019F808E033
:101A6000641CE4B2FA2C04D905F04CF90120BDE85D
:101A7000F0812946304605F053F80028F0D1394668
:101A8000304604F0F1FF0020F1E70000000C0140B7
:101A90009020401EC0B20028FBD1704710B50B4CFF
:101AA00001202070032001F09BF902E0142008F0CF
:101AB0002FF90420FFF7A8FD0028F7D000202070A0
:101AC0006068BDE8104008F0B5B90000940100203E
:101AD00010B540F2026006F0E7FD40F2046006F047
:101AE000E3FD40F2036006F0DFFD48F2200303222D
:101AF0004821094804F0C2FF4FF4744303224821EF
:101B0000064804F0BBFF0322BDE810404FF4806399
:101B10004821034804F0B2BF00080140000C014016
:101B2000001001402DE9F04780468946484600F004
:101B300031FC002818D149461DA001F063FE214C5C
:101B40000026A665A9F103091F4D0127B9F1090F68
:101B50000AD2DFE809F00B0909090D0905101E007A
:101B60000420287084F86060BDE8F0872F70FBE7E0
:101B700002202870F8E7FEF7FFFD0028F4D12E7050
:101B80006F7067804046FFF7F1F8BDE8F047FEF759
:101B90004DBEA08C10B1012802D002E0A78400E065
:101BA000A68498F80000401C88F80000DCE70000DC
:101BB0004B65795F4F7065726174652025640D0A0D
:101BC0000000000098AA00208C0100202DE9F047B9
:101BD00007468946484600F0DDFB002814D14E4CEC
:101BE0000025A5654D4E4FF00108B9F10C0F0BD241
:101BF000DFE809F00A0C0A686344366F2106768430
:101C00000420307084F86050BDE8F087FEF7B4FD22
:101C10000028F9D1A088B4F848108842F4D9218866
:101C20000229F1D0401EA0803846FFF79FF8BDE89A
:101C3000F047FEF719BFFEF79FFD0028E4D1A0880A
:101C4000B4F846108842DFD221880229DCD0401C3B
:101C5000A0803846FFF78AF8BDE8F047FEF704BFDA
:101C60002088032802D2401C208000E025803846CE
:101C7000FFF77CF8BDE8F047FEF7B6BDE088002826
:101C8000C2D04FF48071032803D200F10100E0803C
:101C90000CE007D12088022801D0E18006E0A4F8FA
:101CA000068003E0884201D1A4F806803846FFF799
:101CB0005DF8BDE8F047FEF7F7BE0320307084F80A
:101CC0006050A1E7FFF7A6FB00289DD186F80080B1
:101CD0009AE7FEF75DFD002896D10220307093E769
:101CE000FEF74AFD00288FD1357075706580384643
:101CF000FFF73CF8BDE8F047FEF756BDA08C10B1E9
:101D0000012803D003E0A4F8248000E0A5843878FB
:101D1000401C387078E7000098AA00208C01002051
:101D20002DE9F04780468946484600F033FB0028FD
:101D300017D13B4C012600253A4FB9F10C0F10D2B8
:101D4000DFE809F00F1313271B1313341306425750
:101D50000420207087F86050788820B1012800D1D5
:101D60006670BDE8F0876570FBE7788818B10128D8
:101D7000F7D16670F5E76570F3E70320207087F808
:101D80006050788818B10128EBD16670E9E765707A
:101D9000E7E7FFF73FFB0028E3D12670788818B10A
:101DA0000128DED16670DCE76570DAE7FEF7F0FC4B
:101DB0000028D6D102202070788818B10128D0D10F
:101DC0006670CEE76570CCE7FEF7D6FC0028C8D178
:101DD0002570788850B100F0F0007880657040463A
:101DE000FEF7C4FFBDE8F047FEF720BD7E806670B9
:101DF000F5E7B88C10B1012802D002E0BE8400E003
:101E0000BD84788810B1012802D002E0657000E03E
:101E1000667098F80000401C88F80000A1E70000F8
:101E20008C01002098AA00202DE9F0410746884641
:101E3000404600F0AFFA002814D11B4D0022AA65DD
:101E4000A8F10208194C0126B8F10A0F0AD2DFE8FE
:101E500008F00B090909090D0905101E042020705E
:101E600085F86060BDE8F0812270FBE702202070F9
:101E7000F8E7FFF7CFFA0028F4D12670A670AE81FC
:101E80003846FEF773FFBDE8F041FFF701BBA88CB1
:101E900010B1012802D002E0AE8400E0AA843878B4
:101EA000401C3870DEE7000098AA00208C0100205A
:101EB0002DE9F04780468946484600F06BFA002835
:101EC00013D1304C0026A66501272F4DB9F10C0F18
:101ED0000BD2DFE809F00A0C280A350A0A2E1A0686
:101EE0003A480420287084F86070BDE8F087E089E3
:101EF000B4F848108842F8D9401EE0814046FEF709
:101F000035FFBDE8F047FFF7E3BAE089B4F84610C3
:101F10008842EAD2401CE0814046FEF727FFBDE838
:101F2000F047FFF7D5BAFEF727FC0028DDD12E7069
:101F3000DBE7FEF72DFC0028D7D102202870D4E77C
:101F40000320287084F86070CFE7FFF763FA002859
:101F5000CBD12F70AE70A6814046FEF707FFBDE8DB
:101F6000F047FFF795BAA08C10B1012802D002E02B
:101F7000A78400E0A68498F80000401C88F80000C0
:101F8000B3E7000098AA00208C0100202DE9F0475B
:101F900080468946484600F0FDF9002817D1384CA4
:101FA00001250026374FB9F10C0F10D2DFE809F0F8
:101FB0000F1327131B13133013063A5204202070FB
:101FC00087F86050B88920B1012800D1A570BDE81C
:101FD000F087A670FBE7B88918B10128F7D1A57082
:101FE000F5E7A670F3E70320207087F86050B88902
:101FF00018B10128EBD1A570E9E7A670E7E72670D4
:10200000B88918B10128E2D1A570E0E7A670DEE733
:1020100002202070B88918B10128D8D1A570D6E760
:10202000A670D4E7FFF7F6F90028D0D12570B8895B
:1020300010B1012805D008E0BD81A570FFF728FA8E
:1020400003E0BE81A670FFF723FA4046BDE8F047E3
:10205000FEF78CBEB88C10B1012802D002E0BD841E
:1020600000E0BE84B88910B1012802D002E0A67059
:1020700000E0A57098F80000401C88F80000A6E772
:102080008C01002098AA00202DE9F04781460E46D9
:10209000304600F07FF9002819D1184D8246C5F866
:1020A00058A0314616A001F0ADFBB61E1B4C01270F
:1020B0004FF00208092E0AD2DFE806F00B0E0909DC
:1020C0000909090510000420207085F86080BDE82A
:1020D000F08784F800A0FAE72770F8E7FEF758FBCE
:1020E0000028F4D184F80080E770AF824846FEF7FC
:1020F0003DFEBDE8F047FFF70BBA000098AA0020AC
:1021000075696E7431365F74094B65795F4F706520
:10211000726174652025640D0A0000008C010020A6
:102120002DE9F04704468946484600F033F9002877
:102130002DD13A4D0026AE65394F3A484FF001088F
:10214000B9F10B0F23D2DFE809F022362124220651
:10215000582247222700FEF71BFB002817D1E88AE8
:10216000002814D0032805D2401CE8822078401CA7
:10217000207004E0A5F816802078401C20702046CE
:10218000FEF7F4FDBDE8F047FFF7EAB93E70BDE8A1
:10219000F08787F80080FAE7FEF7FAFA0028F6D110
:1021A00002203870FE70AE822046FEF7DFFDBDE8EB
:1021B000F047FFF7ADB900880028E8D0A88BB5F844
:1021C00048108842E3D9401EA8832046FEF7CEFD82
:1021D000BDE8F047FEF748BC00880028D7D0A88BA0
:1021E000B5F846108842D2D2401CA8832046FEF79C
:1021F000BDFDBDE8F047FEF737BC00880028C6D01B
:10220000688B40B1002068832046FEF7AFFDBDE833
:10221000F047FEF7E9BA0120F5E7000098AA002090
:102220008C010020E40000202DE9F04780468A461A
:10223000504600F0AFF8002819D1394C012500268E
:10224000384F4FF00209BAF10C0F10D2DFE80AF054
:102250000F1327301B131313130639520420207059
:1022600087F86090B88A20B1012800D1E570BDE8F8
:10227000F087E670FBE7B88A18B10128F7D1E5705E
:10228000F5E7E670F3E70320207087F86090B88ADE
:1022900018B10128EBD1E570E9E7E670E7E72670B1
:1022A000B88A18B10128E2D1E570E0E7E670DEE710
:1022B0002570B88A18B10128D9D1E570D7E7E67042
:1022C000D5E7FEF765FA0028D1D184F80090B88AE6
:1022D00010B1012805D008E0BD82E570FFF718F9BC
:1022E00003E0BE82E670FFF713F94046BDE8F04711
:1022F000FEF73CBDB88C10B1012802D002E0BD84CD
:1023000000E0BE84B88A10B1012802D002E0E67075
:1023100000E0E57098F80000401C88F80000A6E78F
:102320008C01002098AA002070B5194800F108051A
:1023300001882980418869808188A980C088E880D7
:1023400000210024002235F81200E040C00712D01E
:1023500032B1012A07D0022A08D0032A09D00AE0A4
:1023600041F0010107E041F0020104E041F0040105
:1023700001E041F00801521CD2B2042AE3D3204606
:1023800007F028FF0021641CE4B20C2CDAD370BDE6
:102390005C0000201249CA8C898C002A02D0012AD4
:1023A00010D012E011B1012902D00EE000207047D8
:1023B0000A2805D0042803D00B2801D0012070473B
:1023C0000020704719B1012903D001207047002077
:1023D00070470B2801D00120704700207047000093
:1023E00098AA002010B5182006F08AFB292006F0D4
:1023F00087FB012006F084FB032006F081FB00240C
:102400000021204607F0E6FE641CE4B20C2CF7D352
:1024100010BD000038B504463E48B0F842103EA05A
:1024200001F0F0F9214649A001F0ECF900200090FC
:10243000FEF7A2F908B1022C6AD0FEF7EBFF08B153
:10244000032C65D0FEF7A4F908B1072C60D0424DEB
:1024500042A0297801F0D6F92878032848D2DFE88D
:1024600000F0021C3200697844A001F0CBF96A78D0
:1024700022B1012A07D0022A3AD109E02146684652
:10248000FFF750FB34E021466846FFF79FFB2FE043
:1024900021466846FFF744FC2AE0AA7822B1012AC7
:1024A00007D0022A24D109E021466846FFF7BCFC88
:1024B0001EE021466846FFF7FBFC19E0214668460E
:1024C000FFF764FD14E0EA7822B1012A07D0022A5E
:1024D0000ED109E021466846FFF7D6FD08E0214607
:1024E0006846FFF71DFE03E021466846FFF79CFEA5
:1024F0002C48006808B901F081FA9DF80000002816
:1025000006D02948012200231102006808F02EFAA3
:1025100038BD000098AA00206469735F7061676528
:102520005F706172616D2E666163655F706C61746E
:10253000655F706172616D2E50616E656C5F53688E
:1025400069656C642025640D0A0000006B657920C4
:1025500025640D0A000000008C0100206469735F8F
:10256000706167655F6E756D2E646973706C6179FB
:102570005F706167652025640D0A00006469735F00
:10258000706167655F6E756D2E4469735F61697216
:102590005F436F6E646974696F6E696E2025640DA8
:1025A0000A000000B8010020040000202DE9F041DD
:1025B00005460C461248002601274188914202D068
:1025C0002E7004B1277042800F2A0ED002EB8200D9
:1025D0004FF6FF7101EA400000F0B0FE011F022932
:1025E00005D82F70002C00D02670BDE8F081401E69
:1025F0000228FAD82E70002CF7D02770F5E70000DB
:10260000AA0100202DE9F04F95B0502101A8FDF757
:1026100022FE45490122CA87002081F8200040F2AD
:1026200001134B814B82C88348848884C884088501
:102630000F274F858A854FF0040CA1F82EC00A861B
:102640004FF47078A1F832808886C886A1F84000DF
:102650004FF00709A1F842904FF01E0AA1F846A0DA
:102660004FF0100BA1F848B0A1F84A00088048804C
:1026700012258D800224CC80088188811C26CE8181
:10268000088248838882CC828D83ADF80420ADF81F
:102690000600ADF80830ADF80A30ADF80C00ADF822
:1026A0000E00ADF81000ADF81200ADF81400ADF852
:1026B0001670ADF81820ADF81AC0ADF81C20ADF8B2
:1026C0001E80ADF82000ADF82200ADF82400098F7F
:1026D000ADF82610ADF82800ADF82A90ADF840A06E
:1026E000ADF842B0ADF84400ADF82C00ADF82E00C6
:1026F000ADF83050ADF83240ADF83400ADF83600EA
:10270000ADF83860ADF83A00ADF83C00ADF83E40A9
:102710000649086088800870502101A800F09AFAE4
:1027200015B0BDE8F08F000098AA00208C010020B1
:10273000FFB50020AD4E96F82010C1F3031201F052
:102740000F03002101250F2A03D1072B01D20121FC
:1027500003E012B9092B00D90121002211B186F83A
:102760002020012071890B0ACCB20021022B01D953
:10277000012102E0032C00D9012140F2011711B11F
:102780007781401CC0B2718A0B0ACCB20021022BA7
:1027900001D9012102E0022C00D9012111B1778277
:1027A000401CC0B2F18B012902D9F283401CC0B297
:1027B000718C0F278B1F092B01D30F2902D9778426
:1027C000401CC0B2B18C012902D9B284401CC0B2F5
:1027D000F18C012902D9F284401CC0B2318D01294B
:1027E00002D93285401CC0B2718D8B1F092B04D2D7
:1027F00005217185401CC0B204E00F2902D97785FC
:10280000401CC0B2B18DC1F3032301F00F040021BD
:10281000012B01D9012102E0062C00D9012111B1BF
:10282000B585401CC0B2F18D072902D9F585401C41
:10283000C0B26F4991E81810C9688DE8181003916B
:102840000021738E6C4634F811C0634503D0491CD7
:10285000C9B20729F7D3072904D14FF470717186E3
:10286000401CC0B2B18E0B0ACCB20021032B01D99F
:10287000012102E00C2C00D9012111B1B286401CCB
:10288000C0B2F18E012902D9F286401CC0B2718C0F
:102890008B1F092B01D30F2902D97784401CC0B2AA
:1028A000318F11B1718C052902D93587401CC0B216
:1028B000B6F84010012903D9A6F84020401CC0B248
:1028C000B6F84210072900D821B90721A6F842100E
:1028D000401CC0B2B6F84010E9B33188032902D9D0
:1028E0003280401CC0B27188012902D97280401C1C
:1028F000C0B2B18819270A39172902D3B780401C02
:10290000C0B2F188B1F5807F05D009B1032902D9A1
:10291000B580401CC0B200213489230AE4B223B13F
:10292000012B05D0022B03D006E02CB1012103E0DE
:102930000CB1032C00D90121012902D13281401CA4
:10294000C0B20021348A230AE4B22BB1012B06D095
:10295000022B04D007E025E02CB1012103E00CB1EB
:10296000022C00D90121012902D13282401CC0B2BF
:10297000B189012902D9B281401CC0B2F1890A395A
:10298000172902D3F781401CC0B2B18A012902D9AC
:10299000B282401CC0B2F18A09B1032902D9F58282
:1029A000401CC0B2B6F8461010390F2904D31E21BE
:1029B000A6F84610401CC0B2B6F84810A1F11003AA
:1029C0000F2B03D2B6F84630994204D31021A6F853
:1029D0004810401CC0B2B6F84A10012903D9A6F825
:1029E0004A20401CC0B204B0F0BD000098AA0020EC
:1029F0004CB3000870B564214C48FDF72CFC4B4CDF
:102A00000025A4F844505021494800F015F94848E1
:102A10000188E1871E2210230126012920D00A34D3
:102A2000A686A57540F2011121802181A58225830A
:102A30006583A583E5830F21218466840421A18415
:102A4000E684510121856585A585E58607212187D5
:102A5000A287E387A4F840500A3C36490D802BE05A
:102A60000A348178A17581882180C18821810189FA
:102A7000A18281896183C189A183018AE183418A1D
:102A80002184818A6184C18AA184018BE184418B84
:102A90002185818B6185C18BA185018C2183418C2E
:102AA000E185818CE186C18C2187A287E387B0F81C
:102AB0004010A4F840100A3CB4F8401001291DD081
:102AC000258065801220A0800222E2802581A581D8
:102AD0001C23E38125826583A582E282A08316A060
:102AE00000F090FEFFF724FE08B100F02DF894F9F5
:102AF0002000002817DAA4F84C6070BD028D2280F7
:102B0000428D6280828DA280C28DE280028E2281FF
:102B1000428EA281828EE281C28E2282028FA282A6
:102B2000408FE082DBE7A4F84C5070BD98AA0020EB
:102B300024040020E40000205061726D5F53617630
:102B4000652025640D0A000000B595B0502101A84C
:102B5000FDF781FB3648818EADF8041090F9161010
:102B6000ADF806100188ADF808100189ADF80A101B
:102B7000818AADF80C10018BADF80E10428BADF8C8
:102B80001020828BADF81220C28BADF81420028C7D
:102B9000ADF81620428CADF81820828CADF81A20C2
:102BA000C28CADF81C20028DADF81E20428DADF810
:102BB0002020828DADF82220ADF82410C18DADF813
:102BC0002610C18EADF82810028FADF82A20828F12
:102BD000ADF84020C28FADF84220B0F840200A384E
:102BE000ADF8442001291DD10188ADF82C10418891
:102BF000ADF82E108188ADF83010C188ADF83210D4
:102C00000189ADF834108189ADF83610C189ADF86D
:102C10003810018AADF83A10818AADF83C10C08AAC
:102C2000ADF83E00502101A800F014F815B000BD29
:102C3000A2AA0020FEE70000054A03E032F8023BAA
:102C400020F8023B491E89B2F8D2012070470000EB
:102C500000FC000870B505460C460E4E03F00CFE55
:102C6000304603F0A9FD70B103F092FD002070BD65
:102C70002988304603F040FD18B103F089FD00209B
:102C800070BDB61CAD1C641EA4B2F1D203F080FD71
:102C9000012070BD00FC000810B514460E4A92F8E1
:102CA00030202270062262700023A370E070087842
:102CB000207148786071082084F880001146204611
:102CC000FEF78CFC010A94F88030A21E995494F807
:102CD0008010641E085510BD98AA002070B51C46CF
:102CE000164B93F830302370102363700023A370C9
:102CF000E070237161714800A071092000EB410070
:102D000084F88000002004E02518135CEB71401C5F
:102D1000C0B2B0EB410FF7D394F88000801EC1B26F
:102D20002046FEF75BFC010A94F88030A21E9954FD
:102D300094F88010641E085570BD000098AA002009
:102D40007047000070B50446062224492046FDF76E
:102D50008DFA78B3214B0621187820B95A78012AC8
:102D600001D1627812B1012802D006E0217027E07B
:102D70009A78012A01D1A27812B1022802D006E085
:102D800021701DE0DA78012A01D1E2782AB1134AD4
:102D900021780525283A11B102E0217010E010B128
:102DA00001290AD00BE0587828B1906A2060908DF4
:102DB000A08005E00FE0257002E0012802D0257018
:102DC000002070BD987820B1906A2060908DA0801E
:102DD000F6E72570F4E7012070BD00008C010020AB
:102DE00030B4044600222A490878002801D1012085
:102DF00008700978072916D2DFE801F01504070AE0
:102E00000D1013004FF4AF720DE04FF4E1720AE0C1
:102E100040F2262207E040F28A2204E040F2EE224D
:102E200001E040F252321A48001F006800282DD1FC
:102E30001848194B082C29D2DFE804F01220170D8E
:102E40000824041C30BC032106F0D4BA30BC002195
:102E5000124806F0CFBA30BC0121184606F0CABAB3
:102E600030BC0221184606F0C5BA30BC0321184612
:102E700006F0C0BA30BC002106F0BCBA30BC01215B
:102E800006F0B8BA30BC022106F0B4BA30BC7047C4
:102E9000840000200034014000040040002C014068
:102EA00030B4044600221D494988012901D001B9E6
:102EB00064221A49091F096800292DD11848194BA5
:102EC000082C29D2DFE804F01220170D0824041C76
:102ED00030BC032106F08EBA30BC0021124806F047
:102EE00089BA30BC0121184606F084BA30BC0221F0
:102EF000184606F07FBA30BC0321184606F07ABAAD
:102F000030BC002106F076BA30BC012106F072BA5E
:102F100030BC022106F06EBA30BC7047840000203D
:102F20000034014000040040002C01400948012108
:102F30004278022A00D141708278022A00D1817041
:102F4000C278022A00D1C170034800214165816521
:102F5000704700008C01002098AA0020084A094B05
:102F600011681B68994209D00748814202D3A0F238
:102F700009101060116811F8010B11607047000012
:102F8000500000204C0000202304002000B5A3B016
:102F90000C48018D012913D000210191408F010AB5
:102FA0008DF804108DF8050002AA01A90D20FFF785
:102FB00073FE054800231A4602A9006807F020FBAB
:102FC00023B000BD98AA00202400002000B5A3B0C3
:102FD0000C49088D012813D0002001908DF80400C1
:102FE00091F83C008DF8050002AA01A90E20FFF718
:102FF00053FE054800231A4602A9006807F000FBAB
:1030000023B000BD98AA00202400002070B540F233
:10301000026005F049FB40F2046005F045FB124CEC
:10302000422303221021204603F028FD0F4D0F23D9
:1030300003221021284603F021FD0221204603F03F
:1030400013FD0121284603F00FFD0221284603F05D
:103050000BFD0421284603F007FD2846BDE870401B
:10306000082103F001BD00000008014000100140EC
:1030700030B40346224A2348062B3ED2DFE803F051
:10308000030E17222B3421B130BC1021104603F05F
:10309000EDBC30BC1021104603F0E6BC19B130BCC9
:1030A000022103F0E3BC30BC022103F0DDBC21B1FE
:1030B00030BC0221104603F0D9BC30BC02211046BE
:1030C00003F0D2BC19B130BC082103F0CFBC30BC36
:1030D000082103F0C9BC19B130BC012103F0C6BC02
:1030E00030BC012103F0C0BC19B130BC042103F095
:1030F000BDBC30BC042103F0B7BC30BC704700003D
:10310000000801400010014013B5334C9DF8000049
:103110002178814205D0012840D000210846FFF7E0
:10312000A7FF61789DF80100814205D001283AD0BF
:1031300000210120FFF79CFFE1789DF80300814208
:1031400005D0012834D000210220FFF791FF21791A
:103150009DF80400814205D001282ED000210320D3
:10316000FFF786FF61799DF80500814205D00128AF
:1031700028D000210420FFF77BFFA1789DF80200F2
:10318000814205D0012822D000210520FFF770FFE1
:1031900000982060BDF80400A0801CBD0121002023
:1031A000FFF766FFBDE701210846FFF761FFC3E7B0
:1031B00001210220FFF75CFFC9E701210320FFF78F
:1031C00057FFCFE701210420FFF752FFD5E7012188
:1031D0000520FFF74DFFDBE77100002070B50024EC
:1031E00003F06AFD8020FEF7EBFBFEF71FFCF520E5
:1031F000FEF7E6FBFEF71AFC012006F089FD03F05E
:103200005BFD8120FEF7DCFB641CA4B2FEF70EFC24
:10321000642C01D00028EFD10120FEF79BFB04466F
:103220000120FEF797FB05460020FEF793FB03F015
:1032300069FD45EA042020F00300FDF73DF99FED0C
:10324000081B53EC112BFDF7C5F89FED071B53EC42
:10325000112BFDF7B9F8FDF768F900EE100A70BD03
:103260007644CF7701405F3F000000000000184027
:1032700070B5002403F020FD8020FEF7A1FBFEF7CF
:10328000D5FBF320FEF79CFBFEF7D0FB012006F0F8
:103290003FFD03F011FD8120FEF792FB641CA4B2F8
:1032A000FEF7C4FB642C01D00028EFD10120FEF70B
:1032B00051FB04460120FEF74DFB05460020FEF7BA
:1032C00049FB03F01FFD45EA042020F00300FDF751
:1032D000F3F89FED081B53EC112BFDF77BF89FEDE6
:1032E000071B53EC112BFDF76FF8FDF71EF900EEED
:1032F000100A70BD619FC6DE07F7653FCDCCCCCC10
:10330000CC6C4740FFF7B4BF10B5FEF7AFFABDE88D
:103310001040AFF3008010B503F0CEFC8020FEF724
:103320004FFBFEF783FBFE20FEF74AFBFEF77EFB1A
:10333000044603F0E7FC204610BD000010B51F490D
:10334000B1F93A101D4C00F10A021346B4F93A40A3
:103350000A34914203DC844201DB002010BD00F1FD
:103360001E02994203DD914201DA012010BD00F1F5
:103370003203914203DB994201DA022010BD9942E7
:1033800001DB032010BD0D49B1F93A101E31844212
:1033900003DA814201DD042010BD084AB2F93A2067
:1033A0003232814203DC824201DD052010BD8242BF
:1033B00001DC062010BD002010BD000098AA0020EE
:1033C00001461648082928D2DFE801F02704090E33
:1033D00013181D224FF4C872002106F00BB84FF4E9
:1033E000FA72002106F006B84FF41672002106F0BA
:1033F00001B84FF42F72002105F0FCBF4FF4487262
:10340000002105F0F7BF4FF46172002105F0F2BF13
:103410004FF47A72002105F0EDBF7047000C0040B8
:1034200070B506461848006800282BD1174C324664
:103430000321204605F0DEFF32460221204605F03A
:10344000D9FF32460021124805F0D4FF324601214F
:10345000204605F0CFFF0F4D32460121284605F0EA
:10346000C9FF32460021204605F0C4FF3246022142
:10347000284605F0BFFF32462846BDE870400321CC
:1034800005F0B8BF70BD000080000020003401408E
:10349000002C0140000400400349098E814201D103
:1034A000012070470020704798AA00200B480D4962
:1034B000B0F84A200A48012A0AD1C27842B90279F2
:1034C00032B9427922B98A88A0F803208A794271F8
:1034D000B0F803208A8040798871704798AA00204C
:1034E00077000020AA01002010B507F0B5FA0128E6
:1034F00003D0BDE8104006F015BF10BD82B01D48D6
:10350000016841F4700101601B48016841F001014C
:10351000016001688907FCD5416841F08001416084
:103520000022019202E00199491C01910199502960
:10353000F9D3416841F090014160019202E00199A4
:10354000491C019101995029F9D3416821F00301E7
:1035500041600168094B194001604FF41F0181600F
:10356000016821F4802101604260C26202B005F06E
:1035700019BC000088ED00E000100240FFFFF6FEDD
:1035800010B504F0BFFE0121BDE81040880706F029
:1035900033B8000010B5174C1549204606F069F9FC
:1035A00038B1204606F0D2F81349C0B2087006F0D0
:1035B0003DF81249204606F05CF9002816D0104A62
:1035C0000120907051781078814208D2481C5070C8
:1035D000D01C415C2046BDE8104006F0BBB8204638
:1035E000BDE8104040F2073106F026B910BD0000DA
:1035F0000503050000380140CC0500200703070043
:103600008A00002070B5104D104C2946204606F067
:1036100030F928B104F0B6FE2946204606F020F91C
:103620000B49204606F025F908B104F0E7FE0949E8
:10363000204606F01EF9002804D02046BDE8704060
:1036400006F084B870BD000005030500004400408A
:103650000703070000050300FEE710B5002301245F
:10366000022820D006DCD0B1012802D10C704B70AA
:103670008B7010BD03281AD0B0F5807FF9D1012AD4
:1036800019D0042A17D0022A19D0052A17D0032AE4
:1036900001D0062AEDD10B704B708C7010BD0B70F1
:1036A0004B708B7010BD0B704C708B7010BD0B701D
:1036B0004B708C7010BD0C704B708B7010BD0B700C
:1036C0004C708B7010BD00002DE9F0470024DFF82E
:1036D00024A1494D494E4A4FDAF80000012829D06B
:1036E00000220321284605F085FE002211463046BF
:1036F00005F080FE00220121384605F07BFE002205
:103700000221384605F076FE00220321384605F0F6
:1037100071FE00221146284605F06CFE00220121B0
:10372000284605F067FE2846BDE8F0470022022142
:1037300005F060BE00220321284605F05BFE002252
:103740001146304605F056FE00220121384605F0AC
:1037500051FE00220221384605F04CFE00220321D2
:10376000384605F047FE00221146284605F042FE85
:1037700000220121284605F03DFE002202212846B4
:1037800005F038FE4FF47A78404606F0C1FA40F270
:103790008A294A460321284605F02CFE4A46002184
:1037A000304605F027FE4A460121384605F022FE44
:1037B0004A460221384605F01DFE4A460321384696
:1037C00005F018FE4A460021284605F013FE4A4639
:1037D0000121284605F00EFE4A460221284605F042
:1037E00009FE404606F094FA641C5A2CFFF674AFAA
:1037F000BDE8F0878000002000340140002C01402B
:10380000000400400FB4054B10B503A9044A029808
:1038100000F018F810BC5DF814FB000049690008BE
:10382000B401002002E008C8121F08C1002AFAD122
:1038300070477047002001E001C1121F002AFBD130
:10384000704700002DE9FF4F8BB09A460F460546A2
:10385000002606E025280BD052460D9990476D1C96
:10386000761C28780028F5D10FB03046BDE8F08FDF
:103870000024A0460122604900E0044315F8013FFE
:10388000203B02FA03F00842F7D128782E2817D1FE
:1038900015F8010F44F004042A280ED06FF02F020F
:1038A0002878A0F1300109290AD808EB880102EB39
:1038B000410100EB01086D1CF2E757F8048B6D1C09
:1038C000287869283ED006DC0028CDD063280BD0AC
:1038D000642804D136E0732810D075284BD05246A6
:1038E0000D999047761C85E017F8040B8DF80000C1
:1038F00000208DF80100E946012003E057F8049B01
:103900004FF0FF3061074FF0000401D40AE0641C5F
:1039100044450DDA8442FADB19F804100029F6D187
:1039200006E0641C8442FCDB19F804100029F8D17D
:10393000264404E019F8010B52460D999047641E85
:10394000F8D257E001CF4FF00A0B002802DA4042CC
:103950002D2102E0210504D52B218DF82410012111
:1039600003E0E10705D02021F7E70DF120090891D8
:103970000CE00021F9E701CF4FF00A0BF9E75946B7
:10398000FCF7EFFD01F1300209F8012D0028F6D116
:10399000ADEB090000F1200B600701D44FF00108E6
:1039A000D84502DDA8EB0B0000E000208046002493
:1039B00006E009A85246005D0D999047641C761CEC
:1039C00008988442F5DB04E0302052460D99904778
:1039D000761CB8F10001A8F10108F5DC05E019F842
:1039E000010B52460D999047761CBBF10001ABF1DB
:1039F000010BF4DC6D1C34E70928010070B5334D70
:103A0000286B012801D0286810B931480078686017
:103A10002979652003F05FFD2E4E7188A9603088FA
:103A2000E860B0886861F08801280AD002280CD0CC
:103A300003280ED04FF4807290420DD12A820024C8
:103A40000AE001202882012406E0022028820224C4
:103A500002E0032028820324B289AA61F089E86188
:103A6000B38A2B62F08A6862686820B1012813D09B
:103A7000022823D119E0C9B2012003F00DFD297BF2
:103A8000022003F028FD1020696903F03DFDE1B23A
:103A90001C2003F020FD11E0D1B2672003F0FCFCF4
:103AA0006620E96903F030FD08E0D9B2682003F030
:103AB000F3FC95F82410692003F00DFDB6F93A10D7
:103AC000BDE87040182003F01FBD0000B8010020C1
:103AD0008C01002098AA0020A0F130010A2901D30E
:103AE000FF2070473021B0FBF1F201FB120070475C
:103AF00001780A02417811430A02817811430902D0
:103B0000C0780843704700002DE9F04F8DB004469F
:103B10000025DFF8A092217F09F1C000A64E002702
:103B2000DFF898A209F120094FF001080C9008294C
:103B300024D2DFE801F00424466686A6C6E2607F50
:103B4000DFF870B2C0F343000BF1E00B042806D19C
:103B5000584602F022FC0D2801D186F80080607FD3
:103B6000C0F34300052809D1584602F016FC0D2881
:103B7000F9D130780128F6D137700125D8E0607F7F
:103B8000C0F34300042806D10C9802F006FC0D286F
:103B900001D186F80180607FC0F343000528EDD194
:103BA0000C9802F0FAFB0D28E8D170780128E5D1D5
:103BB0007770BAF8000000B9022581A0FFF722FE55
:103BC000B6E0607FDFF8ECB1C0F343000BF1A00B6F
:103BD000042806D1584602F0E0FB0D2801D186F8F2
:103BE0000280607FC0F34300052809D1584602F0E7
:103BF000D4FB0D2804D1B078012801D1B77003257A
:103C000096E0607FDFF8ACB1C0F343000BF1800BAE
:103C1000042806D1584602F0C0FB0D2801D186F8D1
:103C20000380607FC0F34300052809D1584602F0A5
:103C3000B4FB0D287CD1F078012879D1F7700425E8
:103C400076E0607FDFF86CB1C0F343000BF1600BEE
:103C5000042806D1584602F0A0FB0D2801D186F8B1
:103C60000480607FC0F34300052861D1584602F00C
:103C700094FB0D285CD13079012859D13771052585
:103C800056E0607FDFF82CB1C0F343000BF1400B2E
:103C9000042806D1584602F080FB0D2801D186F891
:103CA0000580607FC0F34300052841D1584602F0EB
:103CB00074FB0D283CD17079012839D17771062524
:103CC00036E0607FC0F34300042806D1484602F086
:103CD00064FB0D2801D186F80680607FC0F34300A5
:103CE000052825D1484602F058FB0D2820D1B0798F
:103CF00001281DD1B77107251AE0607FC0F343008A
:103D0000042806D12B4802F048FB0D2801D186F883
:103D10000780607FC0F34300052809D1254802F0E1
:103D20003CFB0D2804D1F079012801D1F771082559
:103D3000207F032808D1607FC0F34300062803D109
:103D40000A2526A0FFF75EFD0C9802F026FB062848
:103D50000DD1484602F021FB062808D1BAF8000030
:103D600048B10021AAF8001021A0FFF74BFD207FE9
:103D7000042802D00DE00121F4E7607FC0F3430086
:103D8000092806D103F0EAFB1E48C0F80080FFF7BF
:103D90009BFC1D4C27602C2204F10C016846FCF7AB
:103DA00041FAD4E9012339462846FEF733FB0DB02A
:103DB000BDE8F08F4C060020E6000020E400002063
:103DC0004B65795F4169725F436F6E646974696FB7
:103DD0006E696E675F4D6F64650D0A004B65795FB4
:103DE0005377697463685F4F6E4F66660D0A000013
:103DF00066756A695F6F725F736875696A692025A5
:103E0000640D0A0080000020B8010020007FFDF74B
:103E1000FBBB0000002005A1074A03E00B5C135424
:103E2000401CC0B20828F9D3704700006E6B78338D
:103E30006C616C7000000000420000202DE9F0472A
:103E40000646DFF8C09009EB06056979A8790002FB
:103E5000EA7910441FFA80F8E878287909294FD0C8
:103E600008DC092918D2DFE801F01A1D2024284BAC
:103E70004B174B000E293DD008DC0A2940D00B29F6
:103E80002DD00C292ED00D2906D12FE0242937D092
:103E9000252935D0282931D00020BDE8F08707F04A
:103EA00073F82DE003F04CFD2AE0287A07F020F9A2
:103EB00026E0287A03F070FC22E000240CE03019A0
:103EC0004844817A0902C07A47182819083007F057
:103ED0003BF8E019001D84B24445F0D310E004F033
:103EE000ADFD0DE0F0B204F03DFD09E0F0B203F0ED
:103EF0006FFB05E0F0B203F00DFC01E0FFF77EFD83
:103F00000120CAE70802002002490860086800286A
:103F1000FCD170472C00002010B56FF0040004F0B5
:103F200043FF094809490068B0FBF1F00849C0B2F5
:103F3000087000EB4002C2EBC0104FF6FF7202EABD
:103F4000C000488010BD00003000002000127A0040
:103F5000CE00002010B50E4890F838400321012013
:103F6000FCF71EFF07210220FCF71AFF082103209F
:103F7000FCF716FF052C05D90521BDE810400420EB
:103F8000FCF70EBF2146BDE810400420FCF77EBFC1
:103F900098AA002010B50A48018841F0200202804A
:103FA0000421052002F028FE0648018821F02002A5
:103FB00002800321BDE81040052002F01DBE000074
:103FC00062000020600000202DE9F0419D4D042199
:103FD000288840F020022A80052002F00DFE9A4E2B
:103FE0009A4C308830B1012825D0022844D00328CB
:103FF00063D082E02088012120F004022280022088
:1040000002F0FAFD2088012120F4806222800A203B
:1040100002F0F2FD2088012140F0020222800846D1
:1040200002F0EAFD2088012120F0200222800520F4
:1040300002F0E2FD61E02088012120F002022280EE
:10404000084602F0D9FD2088012120F480622280F8
:104050000A2002F0D1FD2088012140F004022280D4
:10406000022002F0C9FD2088012120F020022280D8
:10407000052002F0C1FD40E02088012120F002026D
:104080002280084602F0B8FD2088012140F48062B9
:1040900022800A2002F0B0FD2088012120F00402D5
:1040A0002280022002F0A8FD2088012120F02002B9
:1040B0002280052002F0A0FD1FE02088012120F0D1
:1040C00002022280084602F097FD2088012120F498
:1040D000806222800A2002F08FFD2088012120F0DA
:1040E00004022280022002F087FD2088012140F096
:1040F00020022280052002F07FFDF088544F012825
:1041000007D0022826D0032845D0B0F5807F63D0A1
:1041100082E02088012140F008022280032002F082
:104120006BFD2088012120F010022280042002F083
:1041300063FD3888022120F010023A80042002F04A
:104140005BFD2888042120F008022A80032002F069
:1041500053FD61E02088012140F008022280032005
:1041600002F04AFD2088012140F010022280042044
:1041700002F042FD3888022120F010023A8004202B
:1041800002F03AFD2888042120F008022A8003204A
:1041900002F032FD40E02088012140F00802228038
:1041A000032002F029FD2088012140F01002228026
:1041B000042002F021FD3888022140F010023A80EC
:1041C000042002F019FD2888042120F008022A802A
:1041D000032002F011FD1FE02088012140F00802B9
:1041E0002280032002F008FD2088012140F0100207
:1041F0002280042002F000FD3888022140F01002E5
:104200003A80042002F0F8FC2888042140F00802DB
:104210002A80032002F0F0FCB0884FF6FF7100EB1B
:10422000800001EA4000002100B2FDF7C3F8094810
:10423000018841F020020280BDE8F0410321052001
:1042400002F0DABC6200002098AA00205C00002086
:104250005E000020600000202DE9F0419C4D9D4C47
:104260002888218800280AD021460128098821F0C1
:10427000020224D0022840D003285CD078E021F04C
:10428000040222800121022002F0B6FC20880121D4
:1042900020F4806222800A2002F0AEFC20880121F6
:1042A00040F002022280084602F0A6FC208801218C
:1042B00020F020022280052002F09EFC58E001211F
:1042C0002280084602F098FC2088012120F48062B8
:1042D00022800A2002F090FC2088012140F0040294
:1042E0002280022002F088FC2088012120F0200298
:1042F0002280052002F080FC3AE00121228008465D
:1043000002F07AFC2088012140F4806222800A2099
:1043100002F072FC2088012120F004022280022099
:1043200002F06AFC2088012120F020022280052072
:1043300002F062FC1CE001212280084602F05CFCD5
:104340002088012120F4806222800A2002F054FC9F
:104350002088012120F004022280022002F04CFC7F
:104360002088012140F020022280052002F044FC38
:10437000E888594E594F012807D0022826D0032833
:1043800045D0B0F5807F63D082E02088012140F0E5
:1043900008022280032002F02FFC2088012120F057
:1043A00010022280042002F027FC3088022120F035
:1043B00010023280042002F01FFC3888042120F013
:1043C00008023A80032002F017FC61E020880121F6
:1043D00040F008022280032002F00EFC2088012118
:1043E00040F010022280042002F006FC30880221F6
:1043F00020F010023280042002F0FEFB38880421F5
:1044000020F008023A80032002F0F6FB40E020880A
:10441000012140F008022280032002F0EDFB2088F9
:10442000012140F010022280042002F0E5FB3088D8
:10443000022140F010023280042002F0DDFB3888B7
:10444000042120F008023A80032002F0D5FB1FE08F
:104450002088012140F008022280032002F0CCFBDA
:104460002088012140F010022280042002F0C4FBC9
:104470003088022140F010023280042002F0BCFBA0
:104480003888042140F008023A80032002F0B4FB8F
:10449000B5F93A000121FCF78DFF11490889421C4A
:1044A0000A81322804D30878C043087000200881AC
:1044B000087800280AD00B48018841F020020280C9
:1044C000BDE8F0410321052002F096BBBDE8F08174
:1044D00098AA00205C0000205E00002062000020FE
:1044E00064010020600000202DE9F047714E708AC1
:1044F000411C7182322804D37079C043707100204E
:104500007082002400256C4F384697F92010B0F8CF
:104510004C0019B1012805D050B10BE0012809D198
:10452000072407E00724002900DA4942CDB201E060
:1045300097F82050B7F84E00DFF88081DFF88091BF
:10454000E8BB707950B31CB921460120FCF79EFCF2
:10455000072C03D121460120FCF722FC294602202A
:10456000FCF794FC00210320FCF790FC02210420BE
:10457000FCF716FCB8F80000012140F08002A8F812
:104580000020072002F038FBB9F80000032140F0BA
:104590002002A9F80020052002F02EFB707970B9E6
:1045A00008210120FCF7FCFB29460220FCF76EFCE9
:1045B00000210320FCF76AFC0221042000E015E042
:1045C000FCF7EEFBB8F80000012140F08002A8F8EB
:1045D0000020072002F010FBB9F80000032140F092
:1045E0002002A9F80020052002F006FBB7F84E00D3
:1045F00001285CD1707950B31CB921460120FCF729
:1046000045FC072C03D121460120FCF7C9FB2946B4
:104610000220FCF73BFC00210320FCF737FC0221C1
:104620000420FCF7BDFBB8F80000012140F0800237
:10463000A8F80020072002F0DFFAB9F800000321F3
:1046400040F02002A9F80020052002F0D5FA707988
:1046500000282CD11CB921460120FCF717FC072C9F
:1046600003D121460120FCF79BFB08210220FCF727
:1046700097FB00210320FCF709FC02210420FCF732
:104680008FFBB8F80000012140F08002A8F800205C
:10469000072002F0B1FAB9F80000032140F020022F
:1046A000A9F80020BDE8F047052002F0A5BABDE852
:1046B000F08700006401002098AA00205C00002020
:1046C0006000002010B5FCF731FABDE8104002F0A0
:1046D0007FBA000010B50E4890F822400221012058
:1046E000FCF75EFB07210220FCF75AFB08210320A0
:1046F000FCF756FB052C05D90521BDE81040042028
:10470000FCF74EBB2146BDE810400420FCF7BEBBC1
:1047100098AA00200448018841F002020280042186
:10472000012002F069BA00006200002010B51048B4
:10473000018841F0020202800421012002F05CFAAB
:104740000C484FF6FF71C08900EB800001EA400081
:10475000002100B2FCF72EFE0748018841F020023C
:1047600002800321BDE81040052002F045BA000098
:104770006200002098AA00206000002010B51448B4
:10478000018841F0020202800421012002F034FA83
:104790001048B0F93A000121FCF70CFE0E49488997
:1047A000421C4A81322804D34878C0434870002014
:1047B0004881487800280AD00848018841F0200242
:1047C00002800321BDE81040052002F015BA10BD9B
:1047D0006200002098AA00206401002060000020F0
:1047E0000448018841F0010202800421002002F007
:1047F00003BA00006200002070B56548018841F0EE
:10480000010202800421002002F0F6F9614D624E9F
:10481000624CE88A012804D002281BD0032832D039
:1048200049E02088012140F008022280032002F0A4
:10483000E3F92088012120F010022280042002F0F8
:10484000DBF93088022120F010023280042002F0CF
:10485000D3F930E02088012140F0080222800320B3
:1048600002F0CAF92088012140F0100222800420C1
:1048700002F0C2F93088022120F0100232800420B8
:1048800002F0BAF917E02088012140F008022280E6
:10489000032002F0B1F92088012140F010022280AB
:1048A000042002F0A9F93088022140F01002328081
:1048B000042002F0A1F93A480088012855D1688BFC
:1048C000F8B92088012120F004022280022002F0A1
:1048D00093F92088012120F4806222800A2002F0CE
:1048E0008BF92088012140F002022280084602F064
:1048F00083F92088012120F020022280052002F087
:104900007BF9688B01281FD12088012120F0020249
:104910002280084602F070F92088012120F480628C
:1049200022800A2002F068F92088012140F0040268
:104930002280022002F060F92088012120F020026C
:104940002280052002F058F9A88B002100EB80009E
:10495000400000B2FCF72EFD1248018841F0200211
:1049600002800321052002F047F907210120FCF70E
:1049700017FA07210220FCF713FA07210320FCF79E
:104980000FFABDE8704007210420FCF709BA0000C7
:104990006200002098AA00205E0000205C00002039
:1049A000E4000020600000202DE9F0414A4D042180
:1049B000288840F001022A80002002F01DF9474FAC
:1049C000474C484EF88A012804D0022823D00328F7
:1049D00042D061E02088012140F0080222800320BB
:1049E00002F00AF92088012120F010022280042020
:1049F00002F002F93088022120F0100232800420F7
:104A000002F0FAF82888042120F008022A80032006
:104A100002F0F2F840E02088012140F008022280F4
:104A2000032002F0E9F82088012140F010022280E2
:104A3000042002F0E1F83088022120F010023280D8
:104A4000042002F0D9F82888042120F008022A80E6
:104A5000032002F0D1F81FE02088012140F0080275
:104A60002280032002F0C8F82088012140F01002C3
:104A70002280042002F0C0F83088022140F01002A9
:104A80003280042002F0B8F82888042120F00802BF
:104A90002A80032002F0B0F8B7F93A000121FCF7B0
:104AA00089FC11498889421C8A81322804D388787C
:104AB000C043887000208881887800280AD00B487D
:104AC000018841F020020280BDE8F0410321052069
:104AD00002F092B8BDE8F0816200002098AA0020A0
:104AE0005C0000205E0000206401002060000020C7
:104AF00010B50E4890F82E4004210120FCF750F923
:104B000007210220FCF74CF908210320FCF748F9A3
:104B1000072C05D90521BDE810400420FCF740B959
:104B20002146BDE810400420FCF7B0B998AA002047
:104B30002DE9F041264CE08A411CE182322804D361
:104B4000E079C043E0710020E082224DA88DC0F3DF
:104B5000032600F00F0701210846FCF721F9072181
:104B60000220FCF71DF9B5F85200C0B101282DD183
:104B7000E07938B131460320FCF788F93946042042
:104B8000FCF784F9E079002820D131460320FCF7B6
:104B90007DF9BDE8F04108210420FCF701B9E07976
:104BA00038B131460320FCF771F939460420FCF78F
:104BB0006DF9E079002809D108210320FCF7F0F80D
:104BC0003946BDE8F0410420FCF760B9BDE8F0814A
:104BD0006401002098AA002010B51348808FFCF7CC
:104BE000DEF81249088A421C0A82322804D3087966
:104BF000C04308710020088209790D4849B1018835
:104C000041F0080202800321BDE81040084601F08F
:104C1000F3BF018821F0080202800321BDE81040A3
:104C2000084601F0E9BF000098AA002064010020B6
:104C3000600000202DE9F041A94E7088012878D14C
:104C4000A8A0FEF7DFFDB64D0421288840F0200221
:104C50002A80052001F0D0FF3088B24C30B1012805
:104C600025D0022844D0032864D083E02088012185
:104C700020F004022280022001F0BEFF20880121E2
:104C800020F4806222800A2001F0B6FF20880121F2
:104C900040F002022280084601F0AEFF2088012188
:104CA00020F020022280052001F0A6FF62E020888B
:104CB000012120F002022280084601F09DFF208899
:104CC000012120F4806222800A2001F095FF2088D3
:104CD000012140F004022280022001F08DFF208893
:104CE000012120F020022280052001F085FF41E013
:104CF0002088012120F002022280084601F07CFF7A
:104D00002088012140F4806222800A2001F074FF93
:104D10002088012120F004022280022001F06CFF93
:104D20002088012120F020022280052001F064FF6C
:104D300020E0AEE02088012120F002022280084617
:104D400001F05AFF2088012120F4806222800A208D
:104D500001F052FF2088012120F00402228002206D
:104D600001F04AFF2088012140F020022280052026
:104D700001F042FFF0886C4F012807D0022826D0AE
:104D8000032845D0B0F5807F63D082E020880121E0
:104D900040F008022280032001F02EFF208801212C
:104DA00020F010022280042001F026FF3888022122
:104DB00020F010023A80042001F01EFF2888042110
:104DC00020F008022A80032001F016FF61E020880D
:104DD000012140F008022280032001F00DFF20880D
:104DE000012140F010022280042001F005FF3888E4
:104DF000022120F010023A80042001F0FDFE2888F4
:104E0000042120F008022A80032001F0F5FE40E092
:104E10002088012140F008022280032001F0ECFEEE
:104E20002088012140F010022280042001F0E4FEDD
:104E30003888022140F010023A80042001F0DCFEA4
:104E40002888042120F008022A80032001F0D4FEE3
:104E50001FE02088012140F008022280032001F099
:104E6000CBFE2088012140F010022280042001F0B6
:104E7000C3FE3888022140F010023A80042001F07D
:104E8000BBFE2888042140F008022A80032001F09C
:104E9000B3FEB6F93A000121FCF78CFA2349C88920
:104EA000421CCA81322804D3C878C043C87000208D
:104EB000C881C9781E4849B1018841F020020280AA
:104EC000BDE8F0410321052001F096BE018821F0E4
:104ED00020020280BDE8F0410321052001F08CBED4
:104EE00098AA00206469735F706167655F70617282
:104EF000616D2E666163655F706C6174655F706182
:104F000072616D2E4169725F636F6E646974696F5F
:104F10006E5F737769746368203D3D203100000047
:104F2000620000205C0000205E0000206401002080
:104F30006000002070B5154890F8300000F00F04B4
:104F4000C0F3031500210120FBF72AFF07210220EF
:104F5000FBF726FF092D05D90A3DE9B20320FBF72F
:104F60001FFF03E029460320FBF790FF092C06D919
:104F70000A3CE1B2BDE870400420FBF711BF2146B6
:104F8000BDE870400420FBF781BF000098AA002014
:104F900070B5414EB08A411CB182322804D3B07939
:104FA000C043B0710020B08200210120FBF7F8FE61
:104FB00007210220FBF7F4FE3849087800F00F05BE
:104FC000C0F30314088C01280CD0002862D1B079FA
:104FD000F0B3092C37D9A4F10A00C1B20320FBF7C2
:104FE000DFFE34E0B079C0B1092C05D90A3CE1B24A
:104FF0000320FBF7D5FE03E021460320FBF746FF25
:10500000092D06D9A5F10A00C1B20420FBF7C8FE9C
:1050100003E029460420FBF739FFB079002839D195
:1050200008210320FBF7BCFE092D06D90A3DE9B291
:10503000BDE870400420FBF7B3BE2946BDE87040D0
:105040000420FBF723BF21460320FBF71FFF00E0EE
:105050000BE0092D05D90A3DE9B20420FBF7A0FEBB
:1050600003E029460420FBF711FFB079002811D195
:10507000092C05D90A3CE1B20320FBF791FE03E0BD
:1050800021460320FBF702FFBDE870400821042001
:10509000FBF786BE70BD000064010020C8AA002096
:1050A00010B50E4890F82A4006210120FBF778FE43
:1050B00007210220FBF774FE08210320FBF770FE96
:1050C000052C05D90521BDE810400420FBF768BE7A
:1050D0002146BDE810400420FBF7D8BE98AA002066
:1050E00010B50A4890F84A4005210120FBF758FE08
:1050F00007210220FBF754FE08210320FBF750FE96
:105100002146BDE810400420FBF7C0BE98AA00204D
:10511000034608461146652B1AD009DC012B11D035
:10512000022B11D0102B11D01C2B19D100F060B81C
:10513000662B0FD0672B0FD0682B0FD0692B0FD1A8
:1051400000F010B800F050B900F0BEB800F0A4B9FB
:1051500000F0C4B900F07EB900F012B900F0DCB87C
:10516000704700002DE9F041044688461E4D002797
:105170002F630126EE622E60FDF7D8FE41462046E1
:1051800002F0E8F904466C621849200006D00128B4
:105190000AD002280ED0032819D112E0CF820021B4
:1051A0000120FCF7FDF912E0CE8201210020FCF77E
:1051B000F7F90CE00220C88202210020FCF7F0F988
:1051C00005E00320C88203210020FCF7E9F96C62A6
:1051D0002146692002F07FF9012802D00020BDE8B5
:1051E000F0810120FBE70000B801002098AA002010
:1051F0002DE9F04104468846304D00272F630126F3
:10520000EE622E60FDF792FE4146204602F0A2F9C2
:10521000044602222A486968032311B1022941D1B8
:1052200020E028490F702C8234B1012C0BD0022CC5
:105230000ED0032C36D110E04FF480712982C1804A
:10524000FBF732FC2EE02E82C680FBF72DFC29E016
:105250002A82C280FBF728FC24E02B82C380FBF764
:1052600023FC1FE06C6234B1012C0AD0022C0ED05A
:10527000032C17D111E0C78200210120FCF790F91F
:1052800010E0C68201210020FCF78AF90AE0C28200
:1052900002210020FCF784F904E0C38203210020EE
:1052A000FCF77EF921461C2002F015F9012802D0F6
:1052B0000020BDE8F0810120FBE70000B8010020DC
:1052C00098AA00208C0100202DE9F04104460E46EA
:1052D0000F4D00222A63FDF729FE3146204602F0D9
:1052E00039F9044601262E60EE620A4F686818B943
:1052F000EC603C80FBF778FA022C04D1F888B0F51A
:10530000807F00D1FE80FEF779FB0120BDE8F081AF
:10531000B801002098AA00202DE9F04106468846F1
:10532000144C00272763FDF701FE01252560414647
:10533000304602F00DF906460F48A6B16563858236
:10534000FCF7E6F825620D480023012210210068D1
:1053500005F00CFB3146682002F09EF8012807D0CA
:105360000020BDE8F0818782FCF7D2F82762EAE7E7
:105370000120F6E7B801002098AA002004000020D0
:105380002DE9F04106468846144C00272763FDF7B7
:10539000CDFD012525604146304602F0D9F806468C
:1053A0000F48A6B165638581FCF772F8A5610D48C9
:1053B000002301221021006805F0D8FA3146672049
:1053C00002F06AF8012807D00020BDE8F08187814B
:1053D000FCF75EF8A761EAE70120F6E7B8010020D4
:1053E00098AA0020040000202DE9F04107468846D5
:1053F000154C00262663FDF799FD012525604146E1
:10540000384602F0A5F807461049AFB16563CE866D
:105410004D80FBF70BFAA5600D48002301221021F7
:10542000006805F0A3FA3946012002F035F801289A
:1054300008D00020BDE8F081CE864E80FBF7F6F95B
:10544000A660E9E70120F5E7B801002098AA00204E
:105450000400002070B50E4C0122E262226002F0CE
:105460007BF80546FDF762FD626832B1012A04D17E
:10547000E5610848C581FCF72BF82946662002F053
:1054800043F8012801D0002070BD012070BD00004C
:10549000B801002098AA002070B50E4C00222263AB
:1054A0000126E66202F058F80546FDF73FFD26604A
:1054B000626822B9656108488580FBF7D5FA2946FC
:1054C000102002F021F8012801D0002070BD012039
:1054D00070BD0000B801002098AA002070B5084CEB
:1054E000002222630126E66202F034F805462660B7
:1054F000FDF71CFD65602846FEF780FA012070BDAF
:10550000B80100202DE9F04FA1B00646002396F81F
:10551000058008F105008DF8800030786D468DF823
:10552000000003208DF801004FEA480003248DF8A5
:105530000200F94FDFF8E493F949002228E2F078FD
:10554000112876D00CDC112874D2DFE800F0FB22A1
:10555000414B838D9AC0CAD773E1FAF9F873F7000B
:105560001A2868D009DCA0F112000828ECD2DFE884
:1055700000F0F0EFEEEDECEB61EA64380D28E3D2D9
:10558000DFE800F0EEEDEC585858585858EBEAE9CF
:10559000E800601C00F0FF0C2A5500204C895FEAEF
:1055A000C47A01D1A40704D47C78012C05D1012050
:1055B00003E03C78012C00D101208C7804F00F042A
:1055C00004EB00100CF10104E4B205F80C00DAE180
:1055D000601CC0B22A5591F800C0441CE4B205F822
:1055E00000C0D0E1002097F803C0BCF1010F0AD041
:1055F00097F804C0BCF1010F07D097F805C0BCF1C3
:10560000010F04D004E0012002E0012000E00120AD
:10561000B1F806A04FEA1A2B0AF00F0C0CEB001C95
:105620000CF0FF0C5FEACA5A0BD528B1012806D04E
:1056300007E0D9E0A1E12DE14FF0000C01E04FF0CF
:10564000100C601CC0B205F804B0441CE4B205F8AC
:1056500000C098E1601CC0B22A5591F804C0441CF7
:10566000E4B205F800C08EE1B1F808C0601C4FEA52
:105670001C2AC0B205F804A0441CE4B205F800C01E
:1056800081E10020B1F812C05FEACC7A06D097F829
:1056900000C0BCF1010F0AD1012008E05FEA8C7C58
:1056A00005D597F801C0BCF1010F00D1012004F12C
:1056B000010C0CF0FF0C2A550C7B04F00F0404EBDA
:1056C00000100CF10104E4B205F80C005BE1601C71
:1056D000C0B22A5591F80EC0441CE4B205F800C0CF
:1056E00051E1B1F810C0601C4FEA1C2AC0B205F8A5
:1056F00004A0441CE4B205F800C044E1601CC0B240
:105700002A5591F814C0441CE4B205F800C03AE1EF
:105710000020B1F81EC0BCF1010F27D197F803C0DB
:10572000BCF1010F1DD097F804C0BCF1010F1AD0D5
:1057300097F805C0BCF1010F17D017E047E03CE037
:105740002EE023E002E19BE08DE082E077E06CE078
:1057500061E056E0F0E0E5E0D4E0C9E0BEE0B0E0B2
:10576000A2E0012002E0012000E0012004F1010C90
:105770000CF0FF0C2A558C7D04F00F0404EB001094
:105780000CF10104E4B205F80C00FCE0601CC0B2AE
:105790002A5591F820C0441CE4B205F800C0F2E09C
:1057A000B1F83AC0601C4FEA1C2AC0B205F804A048
:1057B000441CE4B205F800C0E5E0601CC0B22A5504
:1057C00091F83CC0441CE4B205F800C0DBE0B1F83D
:1057D0000AC0601C4FEA1C2AC0B205F804A0441C91
:1057E000E4B205F800C0CEE0B1F812C0601C4FEA88
:1057F0001C2AC0B205F804A0441CE4B205F800C09D
:10580000C1E0601CC0B22A5591F81EC0441CE4B22D
:1058100005F800C0B7E0601CC0B22A5591F822C05C
:10582000441CE4B205F800C0ADE0601CC0B22A55CB
:1058300091F824C0441CE4B205F800C0A3E0601C49
:10584000C0B22A5591F826C0441CE4B205F800C045
:1058500099E0601CC0B22A5591F828C0441CE4B2FB
:1058600005F800C08FE0B1F82CC0601C4FEA1C2A7C
:10587000C0B205F804A0441CE4B205F800C082E000
:10588000601CC0B22A5591F82AC0441CE4B205F845
:1058900000C078E0601CC0B22A5591F83EC0441C9C
:1058A000E4B205F800C06EE0B1F832C0601C4FEA07
:1058B0001C2AC0B205F804A0441CE4B205F800C0DC
:1058C00061E0B1F834C0601C4FEA1C2AC0B205F890
:1058D00004A0441CE4B205F800C054E0601CC0B24F
:1058E0002A5591F836C0441CE4B205F800C04AE0DD
:1058F000601CC0B22A5591F840C0441CE4B205F8BF
:1059000000C040E0601CC0B22A5591F842C0441C5F
:10591000E4B205F800C036E077000020A8010020BE
:1059200098AA0020601CC0B22A5591F846C0441CB9
:10593000E4B205F800C026E0601CC0B22A5591F818
:1059400048C0441CE4B205F800C01CE0601CC0B2B2
:105950002A55B1F84440012C08D199F800401CB1F7
:10596000641E89F8004001E0A1F8442091F844C089
:10597000441CE4B205F800C005E0601CC0B22A5522
:10598000441CE4B22A54F078401CF0705B1CDBB27B
:105990004345FFF4D4AD21466846FBF71FFE030ADA
:1059A0002246641CE1B2AB544A1C68548DF8802036
:1059B000812269463046FAF735FC21B0BDE8F08F08
:1059C00038B50446E078A17800EB012082B20020CF
:1059D00000906B46611D201D00F028F818B9607812
:1059E00040F08000607094F88000801EC1B22046B4
:1059F000FBF7F4FD010A94F88030A21E995494F844
:105A00008010641E08559DF80000074C28B1012243
:105A100000231102206804F0A9FF002301221021B5
:105A2000206804F0A3FF38BD040000202DE9FF47E3
:105A300005460024DFF8E4930127F94E4FF0020AEF
:105A4000A046122A72D00CDC122A30D2DFE802F013
:105A5000F0254969A5C6EFEEEDEC2FEBEA2F2F2FCD
:105A6000E9E8642A77D009DCA2F11302072AECD214
:105A7000DFE802F0F0EFEEEDEC1DEB006E2A6BD0EC
:105A800006DC652A69D0662A68D06D2A0FD150E3FA
:105A90006F2A6FD0702AF9D1C6E3FAF76DFE18B1FC
:105AA000002004B0BDE8F087287808B10124D3E3D2
:105AB0000878012802D050B10124CDE3778089F81D
:105AC000008089F801701846FBF750F9C4E3A6F886
:105AD000028089F8008089F801801846FBF746F9B2
:105AE000BAE3FAF749FE08B10020DAE7287808B1EE
:105AF0000124B1E37088012801D00124ACE30878C7
:105B000038B1012805D0022803D0032801D0012490
:105B1000A2E389F80080087830801846FBF726F960
:105B20009AE3FAF729FE10B10020BAE732E22878AA
:105B300018B101281FD001248EE37088012801D0FC
:105B4000012489E30878012809D0022807D0032816
:105B500005D0012480E395E2FDE2BAE2D8E289F8BB
:105B600000800878297840EA0120F0801846FBF789
:105B7000FDF871E343E37088012801D001246BE351
:105B8000087808B1012467E389F800804FF4807039
:105B9000F0801846FBF7EAF85EE3FAF7EDFD08B18E
:105BA00000207EE7287808B1012455E37088012899
:105BB00001D0012450E30878B6F8482090420BD376
:105BC000B6F84620904207D889F800800878B0805F
:105BD0001846FBF7CBF83FE301243DE3FAF7CCFD91
:105BE00008B100205DE77088012801D0012433E36B
:105BF0007089BAEB102F51D1C0B2012805D002280C
:105C00001ED0032834D0012426E32878012801D0AF
:105C1000012421E3087801280BD050B101241BE3B3
:105C20006CE123E1FEE0DBE0B8E07CE05AE037E045
:105C30000FE340F4807030811846FBF797F80BE3D0
:105C40002878022807D0012406E309E2F5E1E6E11D
:105C5000D7E1C8E1B8E10878012802D008B10124F1
:105C6000FAE240F4007030811846FBF77FF8F3E267
:105C70002878032801D00124EEE2087838B1012801
:105C800005D0022803D0032801D00124E4E240F427
:105C9000407030811846FBF769F8DDE20124DBE251
:105CA000FBF7B8FB08B10020FBE6287808B1012417
:105CB000D2E20878012802D050B10124CCE2B781A9
:105CC00089F8007089F802701846FBF74FF8C3E2B4
:105CD000A6F80C8089F8007089F802801846FBF756
:105CE00045F8B9E2FBF796FB08B10020D9E6287821
:105CF00008B10124B0E2B089012801D00124ABE24F
:105D00000878B6F8482090420BD3B6F84620904267
:105D100007D889F800700878F0811846FBF726F854
:105D20009AE2012498E2FBF775FB08B10020B8E67F
:105D3000B089012801D001248EE2708ABAEB102FBD
:105D40002AD1C0B2012803D0022813D0012483E253
:105D50002878012801D001247EE20878012802D0A9
:105D600008B1012478E240F4807030821846FAF7D6
:105D7000FDFF71E22878022801D001246CE2087846
:105D8000012802D008B1012466E240F4007030829C
:105D90001846FAF7EBFF5FE201245DE2FAF7F8FC40
:105DA00008B100207DE6287808B1012454E2087883
:105DB000012802D050B101244EE2B78289F800A038
:105DC00089F803701846FAF7D1FF45E2A6F8148067
:105DD00089F800A089F803801846FAF7C7FF3BE26C
:105DE000FAF7D6FC08B100205BE6287808B1012458
:105DF00032E2B08A012801D001242DE2087801287E
:105E000005D0022803D0032801D0012424E2F08227
:105E100089F800A01846FAF7A9FF1DE28C010020BE
:105E200098AA0020287808B1012415E208780F22EA
:105E3000B2EB101F0BD100F00F00C01F082804D8D0
:105E40001F70087886F8200006E2012404E20209A7
:105E500001D0012400E200F00F00092804D81F70CF
:105E6000087886F82000F7E10124F5E1FAF784FCD0
:105E700008B1002015E6287828B101280DD00228A5
:105E80000BD00124E8E1087808B10124E4E11F7097
:105E9000A6F80A80A6F80880DEE10878012805D077
:105EA000022816D0032814D00124D5E1F08B08B1C4
:105EB0000124D1E11F7008782A7840EA022070811D
:105EC000308900F47F403081097840EA0120308138
:105ED000C2E1F08B08B9708A08B10124BCE11F70DF
:105EE00008782A7840EA02207081308900F47F40E7
:105EF0003081097840EA01203081ADE1FBF78AFA70
:105F000008B10020CDE5287828B102280DD001285D
:105F10000BD00124A0E1087808B101249CE11F7096
:105F2000A6F81280A6F8108096E10878012803D020
:105F300002281CD001248FE1708948B1A0F580723D
:105F4000013A05D0A0F50072013A01D0012483E1A5
:105F50001F7008782A7840EA02207082308A00F4A4
:105F60007F403082097840EA0120308274E17089F4
:105F700008B1012470E11F7008782A7840EA0220F5
:105F80007082308A00F47F403082097840EA012034
:105F9000308261E1FAF7FCFB08B1002081E5287846
:105FA00008B1012458E1087818B1012805D001246E
:105FB00052E11F70A6F81E804EE1708908B10124DD
:105FC0004AE11F70F78347E1287808B1012443E1D3
:105FD0000878052803D90F2801D001243CE11F705F
:105FE0000878708438E1287808B1012434E1087811
:105FF00018B1012801D001242EE11F700878B08467
:106000002AE1287808B1012426E1087818B101288E
:1060100001D0012420E11F700878F0841CE1287869
:1060200008B1012418E1087818B1012801D0012431
:1060300012E11F70087830850EE1287818B1012828
:1060400001D0012408E10878401E052806D81F70F9
:106050000878297840EA0120B085FDE00124FBE0C2
:10606000287808B10124F7E00878052803D90F281B
:1060700001D00124F0E01F700878297840EA01205F
:106080007085E9E00878297840EA01217E4890E8A7
:106090002410C0688DE82410039000206A4632F86E
:1060A00010508D4203D0401CC0B20728F7D30728F8
:1060B0000CD0708E884208D01F7071867348012200
:1060C00000231103006804F051FCC5E0641CE4B235
:1060D000C2E0287838B101280DD002280BD003285F
:1060E00009D00124B8E0087808B10124B4E01F7099
:1060F000A6F83480B0E00878401E0B2806D81F7040
:106100000878297840EA0120B086A5E00124A3E0C0
:10611000287808B101249FE0087818B1012801D03F
:10612000012499E01F700878297840EA0120F08660
:1061300092E0287808B101248EE0087818B101288F
:1061400001D0012488E01F700878297840EA0120F6
:10615000A6F8400080E0287808B101247CE00878A7
:1061600007284AD8C0B31F700878297840EA01216F
:10617000A6F84210480703D4A6F8028089F80180E7
:10618000880703D4A6F80C8089F80280C80703D1D9
:10619000A6F8148089F8038099F80000042805D037
:1061A000032803D03A48027812B109E03948FAE7E7
:1061B0004A0705D4890702D480F800A000E00770E0
:1061C000017801290BD1B6F842108A0707D4490794
:1061D00003D480F800A002E00FE080F8008001788E
:1061E000022939D1B6F84210CA0735D1490701D47E
:1061F000077031E080F800802EE001242CE0287840
:1062000008B1012428E00878A0F10A01162909D86C
:10621000B6F84810884203D9A6F846001F701BE064
:10622000012419E0012417E0287808B1012413E0C3
:106230000878A0F10A01162909D8B6F84610884254
:1062400003D2A6F848001F7006E0012404E00124F0
:1062500002E0287818B10124A4B1002021E40878D4
:106260000D4D012802D040B10124F5E7FCF7CAF931
:10627000A6F8447003202870EEE7A6F8448085F85D
:106280000080E9E701200CE45CB300080400002072
:106290008C010020F8AA0020A8010020F8B50446CF
:1062A000E078A17800EB012080B2FF2845D8607922
:1062B000217900EB012086B2FF2E3ED8A079B0EB09
:1062C000460F3AD100200090002514E0A178E07834
:1062D00005EB0121084482B204EB450000F10801FE
:1062E000C01D6B46FFF7A2FB18B9607840F0800034
:1062F00060706D1CEDB2B542E8D394F88000801E4A
:10630000C1B22046FBF76AF9010A94F88030A21E58
:10631000995494F88010641E08559DF80000074CAD
:1063200028B1012200231102206804F01FFB002382
:1063300001221021206804F019FBF8BD04000020A0
:10634000024901200870002103F050BB6D000020BD
:106350000121002003F04ABB002206E0835CFF2BF2
:1063600001D001207047521C92B28A42F6D300201D
:10637000704770B504460D4600F07EFA04212046B1
:10638000FFF7EAFF08B1012070BD2946204600F062
:106390008FFA00F0FDF9002070BD407FC0F343008C
:1063A000704700002DE9F0470026884F7C68387858
:1063B000401EC5B24FF00108B14601E1607F4109BE
:1063C00009D0A189491C89B2A1814FF6FF7291427F
:1063D00001D3218BA181410904D001291DD00229BB
:1063E00015D1C6E0FA6808FA05F1114210D0A4F8F8
:1063F0000C90A4F80E9020F01E006077A16809B1FF
:1064000020468847607F20F0E00020306077CFE0B2
:1064100020F01E001A306077CAE0FA6808FA05F129
:1064200011425DD0E189B9B1A289238A9A42EED99D
:10643000032900D3032161F344006077A16809B107
:1064400020468847607F20F0E00020306077A4F885
:106450000C90A4F80E90ABE0A189628B91420DD311
:10646000C0F34301092908D020F01E0012306077E4
:10647000A168002901D02046884799E0228B9142EB
:106480000DD3C0F34301082908D020F01E001030BE
:106490006077A168002901D02046884788E0E28A19
:1064A00091420DD3C0F34301062908D020F01E000D
:1064B0000C306077A16800297AD02046884777E0C1
:1064C000A28A914274D3C0F34301042970D020F012
:1064D0001E0008306077A16811B32046884767E046
:1064E000A189628B91420CD320F01E001630607798
:1064F000A16809B120468847607F20F0E0006077FE
:1065000056E0228B91420CD320F01E0014306077AD
:10651000A16809B120468847607F20F0E0006077DD
:1065200046E0E28A91420CD320F01E000E306077E4
:10653000A16809B120468847607F20F0E0006077BD
:1065400036E0A28A91420CD320F01E000A30607718
:10655000A16809B120468847607F20F0E00060779D
:1065600026E020F0E00040306077E089401CE081C8
:106570001EE0FA6808FA05F1114206D020F0E000AA
:1065800020306077A4F80C9012E0A189228A914211
:106590000ED9E189032900D3032161F34400607718
:1065A000A16809B120468847607F20F0E00060774D
:1065B000607F400901D0761CF6B224686D1EEDB2F2
:1065C000002C7FF4FBAE3046BDE8F087D4000020FD
:1065D0002DE9F04100260B4F7C683878401EC5B28B
:1065E00006E020468847A840064324686D1EEDB2A9
:1065F00014B161680029F4D1B968F0434840F860EB
:10660000BDE8F081D400002030B5154B59680C4628
:106610004FF0FF35002802D01A78202A06D92846E4
:1066200030BD814201D1284630BD09680029F8D12A
:106630000460417F21F0E00121F01E011A31417711
:1066400000248481C4810F240482586001F0010079
:106650009968904008439860521CD0B2187030BDC1
:10666000D400002010B5FFF7B3FFBDE81040FFF7DE
:1066700099BE00B5034600F009F85B1E012801D160
:10668000002BF8D1012800D1042000BD00200849CA
:10669000CA68D20701D001207047CA68D20601D566
:1066A00003207047C9684907FBD5022070470000E6
:1066B0000020024000B5034600F00AF85B1E0128E6
:1066C00001D1002BF8D1012800D1042000BD000029
:1066D00000200849CA6CD20701D001207047CA6C5B
:1066E000D20601D503207047C96C4907FBD50220AB
:1066F0007047000000200240F0B504460D462048D7
:10670000204E214F0088B0F5007F26D91F488442D3
:1067100011D23846FFF7ADFF00280BD1306940F0A9
:106720000100306125803846FFF7A3FF316921F071
:1067300001013161F0BD3846FFF7BCFF0028F9D1F7
:10674000306D40F00100306525803846FFF7B2FF1C
:10675000316D21F001013165F0BD3846FFF789FF49
:106760000028F9D1306940F00100306125803846B9
:10677000FFF77FFF316921F001013161F0BD0000B9
:10678000E0F7FF1F002002400000FF0FFFFF070897
:106790000748016941F08001016106490988B1F5A6
:1067A000007F03D9016D41F0800101657047000051
:1067B00000200240E0F7FF1F70B504462A482B4D29
:1067C0002B4E0088B0F5007F36D92A48844217D274
:1067D0003046FFF74EFF002811D1286940F0020033
:1067E00028616C61286940F04000286100BF00BF4B
:1067F0003046FFF73EFF296921F00201296170BD93
:106800003046FFF757FF0028F9D1286D40F002000D
:1068100028656C65E869800700D56C61286D40F0DB
:106820004000286500BF00BF3046FFF743FF296DD9
:1068300021F00201296570BD3046FFF71AFF0028DC
:10684000F9D1286940F0020028616C61286940F0A4
:106850004000286100BF00BF3046FFF70AFF2969EA
:1068600021F00201296170BDE0F7FF1F0020024006
:106870000000FF0FFFFF070809480169094A0B06DE
:10688000094901D542604160084B1B88B3F5007F80
:1068900004D9036D1B0601D54264416470470000B2
:1068A0000020024023016745AB89EFCDE0F7FF1FD1
:1068B000F0B504460D462048204E214F0088B0F523
:1068C000007F26D91F48844211D23846FFF7D1FEF7
:1068D00000280BD1306940F0010030612560384656
:1068E000FFF7C7FE316921F001013161F0BD384683
:1068F000FFF7E0FE0028F9D1306D40F0010030656F
:1069000025603846FFF7D6FE316D21F00101316573
:10691000F0BD3846FFF7ADFE0028F9D1306940F0F0
:106920000100306125603846FFF7A3FE316921F090
:1069300001013161F0BD0000E0F7FF1F00200240BF
:106940000000FF0FFFFF070870B50446064DE1B2D7
:10695000284602F0FFFE0721284602F04CFF0028DF
:10696000F9D0204670BD00000038014002494AF6C7
:10697000AA200860704700000030004002494CF631
:10698000CC40086070470000003000400849094BC7
:1069900045F255521A60DA6802F00102491E01D030
:1069A000002AF8D10AB100207047586001207047D2
:1069B000FFFF0F000030004009490A4B45F25552D5
:1069C0001A60DA6802F00202491E01D0002AF8D1EA
:1069D0000AB100207047C0F30B0098600120704797
:1069E000FFFF0F0000300040024945F2555008609B
:1069F000704700000030004010B50023002205E081
:106A000010F8014B2344DBB2521C92B28A42F7D3F6
:106A1000184610BD00B53120FDF75EF88007030E63
:106A20003020FDF759F800F0030043EA001330204E
:106A3000FDF752F800F00F00184300BD10B50446F2
:106A400000F010F801460020054A05E012F8103069
:106A5000A34203D0401CC0B28842F7D310BD00004F
:106A600030B100080B2070474161704701617047E9
:106A7000002A01D001617047416170472DE9F04360
:106A800001F00F04CD0602D5042A18D014430022C9
:106A90004FF00F0C012707FA02F51D401AD0D0F86D
:106AA000009096000CFA06F829EA080904FA06F89C
:106AB00048EA0908282908D0482908D008E044F005
:106AC0000304C26B1A43C263E1E7456100E005615C
:106AD000C0F80080521C92B2082ADCD3082207FAC0
:106AE00002F51D4016D0D0F80490A2F10806B600B9
:106AF0000CFA06F829EA080904FA06F848EA09082F
:106B0000282902D0482902D002E0456100E0056151
:106B1000C0F80480521C92B2102AE0D3BDE8F08382
:106B20008068084201D00120704700207047C0688B
:106B3000084201D00120704700207047F0B5154C85
:106B4000002801DAE36900E06368C0F30346420D00
:106B5000120185B2C0F301579540032F07D0C2023E
:106B60000CD50322B240934343F0E06209E023F0E6
:106B7000E062636823F0E063636002E0AB4343F0EC
:106B8000E06201B12A43002801DAE261F0BD6260EF
:106B9000F0BD00000000014010B540F2026001F0BD
:106BA00083FD40F20E6001F07FFD084C4FF400734E
:106BB000032218212046FFF761FF231520460322F8
:106BC000BDE810400421FFF759BF00000008014054
:106BD00010B500240021204603F0FCFA641CE4B246
:106BE0000C2CF7D303480021018041808180C180B3
:106BF00010BD00005C0000202DE9F0410746174859
:106C000000F1080601883180418871808188B18057
:106C1000C088F0800025002436F81410F940C80719
:106C200012D034B1012C07D0022C08D0032C09D08B
:106C30000AE045F0010507E045F0020504E045F0F3
:106C4000040501E045F008052946384603F0C2FA7C
:106C5000641CE4B2042CDFD3BDE8F0815C000020AA
:106C600010B5FAF71DFEBDE81040FBF7BBBB0000F6
:106C700070B5104E4FF4806529463046FFF7F4FE9C
:106C80006C002346032210213046FFF7F7FE214611
:106C90003046FFF7E9FEFAF7FBFE29463046FFF7DC
:106CA000E5FEFAF7F5FE29463046BDE87040FFF7ED
:106CB000DBBE0000000C014070B5114D4FF40064C4
:106CC0002346032210212846FFF7D8FE66103146DE
:106CD0002846FFF7CBFE21462846FFF7C7FEFAF706
:106CE000D7FE21462846FFF7BFFEFAF7D1FE314610
:106CF0002846FFF7B9FEBDE87040FAF7C9BE0000AC
:106D0000000C014070B5114D4FF40064234603227E
:106D100010212846FFF7B2FE661031462846FFF7DD
:106D2000A3FE21462846FFF79FFEFAF7B1FE314643
:106D30002846FFF79BFEFAF7ABFE21462846FFF7F1
:106D400095FEBDE87040FAF7A3BE0000000C0140BC
:106D500002F0D4FDFFF786FC142002F0D9FFF9E71A
:106D600086B002F08BFEBA481E21CDE90010002348
:106D70004FF48072B7A1BC4803F0C8FD02F0BAFE20
:106D8000BA4F97F82E0000F00F00FCF719FBFFF741
:106D900067FFAF48243800258562858500F1280407
:106DA0002570C16A806ACDE9040178884FF0010836
:106DB000012801D184F80180B889012801D184F823
:106DC0000280B88A012801D184F80380B7F8420014
:106DD0004FF0020908280CD2DFE800F00B04070787
:106DE0000A0A0A0A84F8009003E084F8008000E0B0
:106DF0002570002603F03EFE0390DFF874A240F6F3
:106E0000B93B04A8FBF79EFFDAF80000012857D130
:106E1000DAF8300060BBDAF83400012803D1FDF75E
:106E200051FCCAF83450DAF8040020B1012820D00F
:106E3000022845D137E0012E03D00126FFF7C8FE16
:106E4000BD65DAF80800012802D02570657037E0CA
:106E5000257084F801808DF810508DF81180BAF8F3
:106E60000C003880BAF81000F880BAF81400B88026
:106E700026E0022E03D00226FFF7AAFEBD65DAF84F
:106E80001800012803D084F80080A57018E084F869
:106E9000008084F802808DF810808DF81280BAF896
:106EA0001C00F8810CE0032E03D00326FFF790FEB0
:106EB000BD65DAF8200001280CD084F80090E57058
:106EC0009DF81000072819D2DFE800F0223E5A761C
:106ED0009110190084F8009084F803808DF81090C8
:106EE0008DF81380BAF82400F882E9E7FFF770FE06
:106EF00057482438C16A806ACDE90401A2E0FDF751
:106F0000E1FB53482438C16A806ACDE9040199E065
:106F1000FD6587F860509DF8110020B1012805D06B
:106F2000022802D10DE0FDF735F88BE0B86D411C69
:106F3000B965584502D3BD6584F80190FDF744F862
:106F400080E0FDF789F97DE0FD6587F860809DF8B8
:106F5000120020B1012805D0022873D10DE0FDF701
:106F6000D9FB6FE0B86D411CB965584502D3BD65CA
:106F700084F80290FDF7DAFB64E0FDF7FFFB61E0C7
:106F8000FD6587F860809DF8130020B1012805D0C9
:106F9000022857D10DE0FDF723FC53E0B86D411CEA
:106FA000B965584502D3BD6584F80390FDF724FC0C
:106FB00048E0FDF7F9FC45E0F86D411CF965B0F5D6
:106FC0007A7F03D9FD6597F8600020709DF8140062
:106FD00020B1012805D0022834D105E0FDF72AFEB2
:106FE00030E0FDF7F9FD2DE0FDF7A4FF2AE0786D14
:106FF000411C7965B0F5FF7F03D37D6597F860008C
:1070000020709DF8150008281CD2DFE800F0040766
:107010000A0D10131619FDF767FA13E0FDF7B8FF14
:1070200010E0FDF785FD0DE0FEF73AF80AE0FDF708
:1070300051FB07E0FCF78EFF04E0FDF759FD01E08E
:10704000FEF74EF80A2103A802F09AFED9E60000E6
:10705000880100204765745F74656D705F68756DA9
:10706000695F7461736B00008D16000898AA002098
:10707000B801002070B5884232D11A4D1A4C4FF435
:107080000076B8B14FF001024FF020012846FFF71B
:10709000EFFC012231462846FFF7EAFC012240219D
:1070A0002046FFF7E5FC2046BDE870400122102194
:1070B000FFF7DEBC002220212846FFF7D9FC002282
:1070C00031462846FFF7D4FC002240212046FFF736
:1070D000CFFC2046BDE8704000221021FFF7C8BC5D
:1070E00070BD0000000C01400008014086B003F0B4
:1070F000C1FC0490002003900025824600278046B2
:10710000DFF8DCB1DFF8DC9199F82E008BF8040091
:10711000B9F82C0000F00F018BF80010000A03D022
:107120000120ABF8020002E00020ABF80200B9F841
:107130002A0090B10F2813D040F2771148434FF640
:10714000FF7101EAC0060A2305AA4FF0FF310020B3
:1071500003F00CFD012806D037E040F2DC56F2E7E0
:1071600000260025EFE70598C00311D55E4800789A
:1071700070B902F083FC5C490A20091DCDE90001C9
:107180000023802259A15E4803F0C0FB02F0B2FC4C
:107190000598C00411D55448407870B902F06EFCCF
:1071A00051490A200831CDE900010023802255A170
:1071B000594803F0ABFB02F09DFC0598C10501D5D1
:1071C0004FF0010AC00600D50025BAF1010F0FD11A
:1071D000394652A0FCF716FB38467F1CFFB2052843
:1071E00006D3FBF7A5FAFBF7AFFC4FF0000A002728
:1071F00026B1701C854201D26D1CADB200243A4804
:107200000C30005DF8B92046FAF7FEF928B1B54216
:1072100008D90020FCF704F928E000252046FBF7F8
:10722000DFFD23E0032C02D12F48007858B9012C50
:1072300003D1B9F80200012802D0022C04D007E0E3
:107240002046FBF7CDFD11E0B9F80C00012802D073
:10725000062C04D007E02046FBF7C2FD06E0B9F893
:107260001400012828D02046FBF71AFE641CE4B263
:10727000082CC4D39BF804000399884203D00390E0
:107280000398FCF79DF808F10108B9F83410080AD2
:10729000C9B201EB4102C2EBC1124FF6FF7101EA24
:1072A0008201884516D34FF00008012808D0022833
:1072B00009D003280AD00DE02046FBF791FDD5E761
:1072C000FBF764FE06E0FBF781FE03E0FBF75EFEE2
:1072D000FBF77CFE142104A802F052FD14E7000025
:1072E0008400002098AA0020940100204B455934C6
:1072F0005F355F626C696E6B5F7461736B00000079
:107300009D1A00084368616E67655F626175645F1E
:107310007461736B000000003D0D000857726974C2
:10732000655F666C61675F74696D65202564200D1B
:107330000A0000001CB54FF4407000F0ABFAF9F7FA
:1073400093FC07480121CDE900100023802205A10C
:10735000074803F0DBFA02F09DFE00201CBD000090
:107360000000002073746172745F7461736B0000BD
:10737000898B0008A2B01C4C1C4E30E000235A1E22
:1073800001A903F017F838B3194D02E0012002F00B
:10739000BFFC28780128F9D1002001AA154B9DF8DF
:1073A000841003E0155C1D54401CC0B28142F9D822
:1073B0001148017001202070FEF7CAFF02E0012091
:1073C00002F0A6FC20780028F9D1FEF7B9FFFCF7FF
:1073D00015FB5A2002F09CFC012002F099FC306859
:1073E0000028F9D0CAE700006C000020240000202B
:1073F0006D000020F404002070000020A2B0234C97
:107400004FF0FF36224D34E09DF8841001A8F9F7C3
:107410007CFC70B31F49012008639DF80500032818
:1074200004D006280CD0102821D115E001A8FEF7C1
:1074300069F800231A4601A9206803F0E1F816E074
:1074400001A8FEF7BDFAFBF771FD00231A4601A95A
:10745000206803F0D5F80AE001A8FEF71FFFFBF74C
:1074600065FD00231A4601A9206803F0C9F8FCF75E
:10747000C5FA0023324601A9286802F09BFF9DF857
:107480000400FCF709F80028F3D0BDE72400002031
:1074900020000020B801002010B502460C46002054
:1074A000114601F069FB012101F066FB002101F0AA
:1074B00063FB012101F060FB44B1012101F05CFBA1
:1074C0000146062003F0ECFD012010BD002101F073
:1074D00053FB0146F5E710B502460C460020114665
:1074E00001F04AFB042101F047FB002101F044FBBD
:1074F000012101F041FB214601F03EFB014606203F
:1075000003F0CEFD012010BD10B502460C46002050
:10751000114601F031FB022101F02EFB002101F0A8
:107520002BFB042101F028FB210E01F025FBC4F305
:10753000074101F021FBC4F3072101F01DFBE1B27B
:1075400001F01AFB0146062003F0AAFD012010BD40
:107550000078704700787047FCF7CABA10B5002071
:10756000012101F009FB0146BDE81040032003F0B2
:1075700097BD000070B500230020144CD4E903210E
:10758000914221D204E0E15C01F0F6FA5B1CDBB22F
:10759000082BF8D3217A01F0EFFA002318255A427C
:1075A000216905EBC202D140C9B201F0E5FA5B1CCA
:1075B000DBB2042BF3D3302101F0DEFA0146BDE843
:1075C00070400D2003F06CBD70BD0000F001002084
:1075D0002DE9F0478CB0044600252C216F4601A808
:1075E000F8F739FE4648006800900021454A161910
:1075F000307A01284CD0444809E004EB010C944453
:10760000435C9CF809C0634542D1491CC9B20829B2
:10761000F3D33E4B717C187A884239D10021182669
:1076200060181044807CC1F1000C06EBCC0C00FA11
:107630000CF00543491CC9B20429F1D30021186993
:10764000A84225D1D3F80CC0DFF8C480ACEB050606
:107650008946302E1FD305F1300AD4451BD070B9AE
:10766000C8F804900BE066181644B67D7E547E5C24
:10767000D8F804C06644C8F80460491CC9B230296F
:10768000F1D33030186130226946284600F00CF9F9
:107690000CB0BDE8F0874FF0300CB6FBFCFA0CFBE9
:1076A0001A6CBCF1000F01D0F6B211E030260FE0E9
:1076B00004EB010C94449CF816C007F801C017F8BD
:1076C00001C0D8F804A0D444C8F804C0491CC9B209
:1076D000B142EDD3304418615869D8F8041088429B
:1076E00003D0012000F03EF802E0002000F03AF85C
:1076F00032466946284600F0D7F8C8F80490C7E734
:1077000048B100080802002042000020F0010020DB
:107710003800002010B50E490844007A002815D121
:107720000C48012101600C48FEF723FE4FF4FA706B
:10773000FCF7EAFBBFF34F8F08480168084A01F4E1
:10774000E06111430160BFF34F8FFEE710BD000001
:107750000802002054000020002000080CED00E08A
:107760000400FA0510B501460020002301F004FAD8
:10777000084C04E0E15C01F0FFF95B1CDBB2082B74
:10778000F8D3217A01F0F8F90146BDE810400E2047
:1077900003F086BCF0010020704730B50446204657
:1077A000002C08D00B0006D0884202D98B188342E7
:1077B00012D2002305E0002030BDCD5CC5545B1C17
:1077C0009BB29342F9D309E08B18851813F8013C5A
:1077D00005F8013C521E92B2002AF5D1204630BD78
:1077E0000021002801D17047491C10F8012B002A04
:1077F000FAD108467047000070B505460E460023D2
:10780000002423480168C1F30221072932D001680E
:10781000C1F3022106292FD00168C1F302210529F5
:107820002DD00168C1F3022104292BD00068C0F3D8
:107830000220032829D04FF4A06000F02BF8022387
:107840000224C3F104008640C4F104010F20C840A3
:1078500010403043000105F1E02181F8000405F0FB
:107860001F01012088406909890001F1E021C1F868
:10787000000170BD0424E4E701230324E1E70223AF
:107880000224DEE703230124DBE70423D9E7000019
:107890000CED00E00249084302490860704700000F
:1078A0000000FA050CED00E02DE9F0410E4690468F
:1078B00000240127204A21490B6843440B608518A6
:1078C000B8F1300F03D008F0030048B32BE006EB0B
:1078D0008400C178827802EB0121407800EB01201E
:1078E00016F8241001EB00212846FEF742FD2D1D5D
:1078F000641CA4B20C2CEAD315E006EB8400C1781A
:10790000827802EB0121407800EB012016F8241068
:1079100001EB00212846FEF72CFD2D1D641CA4B2AE
:10792000B4EB980FE9D3002F03D0BDE8F041FFF787
:1079300021BEBDE8F081000000980008580000203A
:1079400010B5002418A0FFF74BFF82B216A1204605
:1079500001F004F9044616A0FFF742FF82B214A119
:10796000204601F0FBF8044614A0FFF739FF82B26D
:1079700012A1204601F0F2F8044612A0FFF730FFF2
:1079800082B210A1204601F0E9F804460FA0FFF7EB
:1079900027FF82B20DA1204601F0E0F80146BDE8C4
:1079A0001040012003F07CBB7B2270223A220000B1
:1079B0006E6B78336C616C7000000000222C2276B4
:1079C000223A2200312E302E30000000227D0000AD
:1079D0002DE9F04104460F46174EF5683068001D4A
:1079E00001F0C0FF38B9306890F82C1001208840B1
:1079F000316981433161601C07D137B13168BDE81D
:107A0000F041091D0D4801F0E5BF2C443068446089
:107A1000AC4206D23168B06B091DBDE8F04101F0FF
:107A2000C1BF3168706B091D01F0BCFFB06A8442B0
:107A300000D2B462BDE8F081F00000205C0A0020B2
:107A400070B5044602F01AF81D4DA868401CA860E5
:107A5000286810B1686938B10CE02C60A86801286A
:107A600008D100F099F905E02868E16AC06A884207
:107A700000D82C60686A401C68626064E06A01217A
:107A80002A698140114329610E4900EB800001EB16
:107A90008000211D01F09EFF02F02CF8686900288B
:107AA0000CD02868E16AC06A884207D206494FF0C4
:107AB00080500860BFF34F8FBFF36F8F70BD000021
:107AC000F00000208C07002004ED00E010B501F06C
:107AD000D5FF0E4C2068A0B90D4801F055FF0C48A9
:107AE000143001F051FF0A48E06014302061002298
:107AF0001021052002F02CFC206010B105A102F03D
:107B0000D1F8BDE8104001F0F5BF00002C010020C5
:107B1000700A0020546D72510000000070B5124EC2
:107B2000124D1CE002F000FB306820B1002403F08D
:107B30000DF9A4B901E00124F9E701F09FFFF06815
:107B4000C468201D01F00EFFA868401EA860686888
:107B5000401E686001F0CEFF204600F054F86868CF
:107B60000028DFD170BD0000480A0020F00000208E
:107B700030B40B46026C002A0CD0C1681144C160BD
:107B80004468A14201D30168C160C16830BC184695
:107B9000F8F748BB30BC70472DE9F0410446174662
:107BA0000026A56B226C002A10D0C7B1E068F8F758
:107BB00039FBE168206C091AE1602268914202D227
:107BC0006168081AE060022F16D017E02068A8B993
:107BD000606803F013F80646002060600EE0A068BD
:107BE000F8F720FB216CA0680844A0606168884217
:107BF00004D32068A06001E005B16D1E6D1CA56373
:107C00003046BDE8F08110B50446206B01F0A6FFB8
:107C10002046BDE8104001F0A1BF00000749CA6836
:107C20001168002904D00021016019B100207047BB
:107C30000121F9E7D0680068704700002C0100209E
:107C40004FF420410F48420706D0C01D20F0070026
:107C50000C49411AC1F520410B4A106000235360C2
:107C60000144083921F00701103A11604B600B60A4
:107C70000B1A436001604068906050604FF0004014
:107C8000D0607047980A002050010020074E4FF046
:107C90008054074DFFF742FF30680128FAD92C6065
:107CA000BFF34F8FBFF36F8FF4E700008C07002006
:107CB00004ED00E070B51D46049C00290BD0226045
:107CC000E06321640121204602F044FC84F8505016
:107CD0000020A06470BD2460F2E700002DE9F047A9
:107CE000DDE908580A9C81460E4617469A46B900B7
:107CF000A522206BF8F7A8FA206B7F1E00EB870007
:107D000020F00707780705D040F22B3219A11EA0FA
:107D1000FBF778FD00202218315C82F83410315CCA
:107D200011B1401C1028F6D3002684F84360202DA2
:107D300000D31F25E562E5642665201D01F02FFEB6
:107D400004F1180001F02BFE2461C5F12000A061B0
:107D50006462666584F8586052464946384600F0C9
:107D600013FC2060B8F1000F01D0C8F80040BDE856
:107D7000F08700002E2E5C4672656552544F535CAE
:107D80007461736B732E63004572726F723A257360
:107D90002C25640D0A00000070B50024114D04EB81
:107DA000840005EB800001F0EFFD641C202CF6D36D
:107DB0000D4801F0E9FD0C48143001F0E5FD0A48DA
:107DC000283001F0E1FD08483C3001F0DDFD0648B7
:107DD000503001F0D9FD05480349416314318163F6
:107DE00070BD00008C0700200C0A0020F00000206D
:107DF00030B5134900E011460A688242FBD34B6854
:107E00005C18844203D140681844486008460D68F5
:107E100044682318AB420DD1094B103B1B689A42B2
:107E200006D05268224442600A681268026002E08A
:107E3000036000E00260814200D0086030BD0000B5
:107E40005001002070B50024416000610C4D91424A
:107E50000AD8D11A8269914201D301240EE0011D92
:107E6000286901F09FFD09E09A4203D2994201D3AB
:107E7000012403E0011DE86801F094FD204670BD77
:107E80002C01002010B5044601F0F8FDA06B20B1D4
:107E9000002401F02FFE204610BD0124F9E710B5A3
:107EA000044601F0EBFDA06BE16B884201D1012497
:107EB00000E0002401F01EFE204610BD2DE9F34134
:107EC0000F460098846C0026002C05D140F6CE1297
:107ED00016A11BA0FBF796FCA06BE16B884205D3B3
:107EE00040F6CF1211A116A0FBF78CFCA06BE16B42
:107EF00088420CD294F945503A4669462046FFF72D
:107F00004BFE0646681C05D06D1C84F84550304673
:107F1000BDE8FC81606A0028F9D004F1240002F079
:107F2000C7FE0028F3D00126F1E700002E2E5C46A4
:107F300072656552544F535C71756575652E6300AB
:107F40004572726F723A25732C25640D0A00000089
:107F5000F8B505460E461348C068C068C468201DC1
:107F600001F000FDE069012816D1A0692B464119F6
:107F700032462046FFF766FF70B1002003460146F7
:107F800000902A46204602F091FF28B94FF4027271
:107F900005A10BA0FBF736FC616A01B02046BDE8E5
:107FA000F04008472C0100202E2E5C467265655279
:107FB000544F535C74696D6572732E63000000004A
:107FC0004572726F723A25732C25640D0A00000009
:107FD00070B586B02F4E53E00298002803DADDE931
:107FE0000320059990470298002849DB049C6069AA
:107FF00010B1201D01F0B6FC01A800F0A9F805465B
:1080000002980A283CD2DFE800F00505053B273836
:1080100005053B270398A169034601442A462046EB
:10802000FFF710FF00282BD0616A20468847E069DF
:10803000012825D1002000900398A169002342184F
:108040001946204602F032FFD0B940F2213212A187
:1080500017A0FBF7D7FB13E00398A06128B94FF4F2
:108060004E720DA112A0FBF7CDFBA0692B46411962
:108070002A462046FFF7E6FE02E0204601F06EFDAC
:1080800000231A4602A9306802F094F90028A3D10F
:1080900006B070BD2C0100202E2E5C467265655224
:1080A000544F535C74696D6572732E630000000059
:1080B0004572726F723A25732C25640D0A00000018
:1080C000F8B506460D4602F02FF8684600F040F875
:1080D0000446009810B102F039FEF8BD45B9A64239
:1080E00006D802F033FE21463046FFF731FFF8BDD7
:1080F0000C481DB10169096891B10025311B2A4660
:10810000006801F0E1FD02F021FE0028EFD10649F0
:108110004FF080500860BFF34F8FBFF36F8FF8BDF3
:108120000125EBE72C01002004ED00E00748416B3E
:108130000968002905D0416BC968C968496881622E
:1081400070474FF0FF31816270470000F00000205F
:1081500070B5054602F08EFC0446074EB0688442B6
:1081600004D200F00BF80120286001E00020286014
:10817000B460204670BD00002C010020F8B5184EF8
:1081800025E0C0680568C468201D01F0EBFB616A4A
:1081900020468847E069012819D1A0692844A842EF
:1081A00006D960602461211DF06801F0FBFB0EE040
:1081B00000200346014600902A46204602F076FE43
:1081C00028B940F2923207A10CA0FBF71BFBF06824
:1081D00001680029D5D1F0683169F1603061F8BDDE
:1081E0002C0100202E2E5C4672656552544F535C64
:1081F00074696D6572732E63000000004572726FC2
:10820000723A25732C25640D0A0000000848406866
:10821000401C05D040F20F1206A111A0FBF7F2FAA4
:10822000502080F31188BFF34F8FBFF36F8FFEE7AD
:10823000580100202E2E5C4672656552544F535CE7
:10824000706F727461626C655C525644535C41524B
:108250004D5F434D34465C706F72742E63000000B6
:108260004572726F723A25732C25640D0A00000066
:1082700008B56846FFF7D2FC0099FFF721FFFFF72A
:10828000A7FEF6E72DE9F041044601F0F7FB94F96B
:10829000455004F1240613E0A06C38B100212046BB
:1082A000FFF70CFE50B101F02BFE07E0606A48B109
:1082B000304602F0FDFC08B101F022FE6D1E6DB2E9
:1082C000002DE9DC4FF0FF3684F8456001F012FC28
:1082D00001F0D4FB94F9445004F1100709E020693F
:1082E00048B1384602F0E4FC08B101F009FE6D1E09
:1082F0006DB2002DF3DC84F84460BDE8F04101F07C
:10830000F9BB000070B5A2B000200090184C207896
:108310000125002802D002281CD102E001F08EFBCA
:1083200018E00020134901AB134A03E0165C1E5409
:10833000401CC0B20E78B042F8D308788DF88400A3
:1083400001F07CFB25700D4800236A4601A90068F6
:1083500002F01EFA25700098002807D008494FF057
:1083600080500860BFF34F8FBFF36F8F22B070BD96
:108370006D0000206F000020740400202000002009
:1083800004ED00E070B5194801F0E0F9C1B2184BF6
:10839000187858B1174C184A01280BD0022815D06C
:1083A000032821D1BDE8704001F058BBBDE8704002
:1083B00001F054BB002050705078451C557021547A
:1083C00002201870BDE8704001F048BB507880284A
:1083D00004D25078431C5370215401E003201870DC
:1083E000BDE8704001F03ABB70BD000000440040A1
:1083F0006D000020740400206E00002070B5154947
:1084000008780025144C002817D0012814D1A27830
:108410001248B2B112492278895C054601F09AF9F6
:108420000721284601F0E7F90028F9D02078401C00
:108430002070A078401EA07070BDFDF789FF2570E8
:1084400070BD25700D70BDE8704040F2073101F03D
:10845000F3B900006C0000206E00002000440040D2
:10846000F40400202DE9F0410546002601F05CFEF1
:10847000304F386808B9FFF7E3FBF86805424BD185
:1084800075B1083568070BD005F00700C0F108008A
:108490000544680704D0BF2227A131A0FBF7B2F939
:1084A000002D39D07868854236D8224910310846E7
:1084B000046801E0214604466068A84202D22068B0
:1084C0000028F7D13868844226D00E680836206824
:1084D00008606068401B102811D904EB05085FEAAA
:1084E000487004D0EC2214A11DA0FBF78BF9606842
:1084F000401BC8F8040065604046FFF779FC6168DE
:108500007868401A7860BA68904200D2B860F8681B
:10851000014361600020206002F018FC700705D064
:108520004FF4967204A10EA0FBF76CF93046BDE83B
:10853000F0810000400100202E2E5C4672656552DD
:10854000544F535C706F727461626C655C4D656D05
:108550004D616E675C686561705F342E630000007A
:108560004572726F723A25732C25640D0A00000063
:1085700004490868002803D00868026D521C02658F
:1085800008687047F000002024384FF080730362C1
:1085900021F00101C1610449816142606FF0020173
:1085A00040F82019704700000D82000870B588B0AF
:1085B0000346002035A104AE91E83400C96834C6F2
:1085C000079133A106C9CDE9021231A106C9CDE94F
:1085D0000012324C6168C1F38101314A002930D068
:1085E00001292ED002292CD1616801F48031B1F526
:1085F000803F11D052106168C1F3834165682D013D
:1086000001D541F0100165686D0001D541F02001F0
:108610000F290ED2891C13E0E16A01F0804101B1FB
:10862000204A616801F40031B1F5003FE3D15208FE
:10863000E1E7A1F10F052F2D01D8491C00E03F21F2
:108640004A436168C1F3031104AD695C22FA01F188
:108650006568C5F3022502AE755D21FA05F564680B
:10866000C4F3C2241DF8044021FA04F443B1012BE1
:1086700008D0022B08D0032B00D1204608B070BDD3
:108680001046FBE70846F9E72846F7E70000000038
:108690000000000001020304060708090010024060
:1086A00000127A00006CDC02054901EB90110A68A7
:1086B00000F01F030120984002430A607047000049
:1086C00000100240054901EB90110A6800F01F03F9
:1086D0000120984082430A60704700000010024069
:1086E000054901EB90110A6800F01F030120984032
:1086F00002430A6070470000001002401FB5FEF7F9
:1087000073F90320FEF742F94FF47A60FEF754F94B
:10871000FEF72CF9FEF732F94FF000080020039025
:10872000834602908D4C00272760A780DFF830A297
:10873000BAF80A30190ABAF81200020ADEB2C5B253
:108740009AF81E900398B04205D0A7702770677002
:10875000E77027716771012E06D0022E28D0032EF4
:1087600050D0002E7BD0DBE0BAF80C00012807D0F7
:108770002770BAF8222000217848F9F717FFCFE0D8
:10878000AB4500D02770012D0DD1BAF81000A0F52F
:108790008071013908D0B0F5807F07D01123002106
:1087A0006E48F8F743FEBBE02223F8E71123F6E713
:1087B000BAF8020001280CD06770E7702771677162
:1087C00001202070BAF822206449601CF9F7EEFEFF
:1087D000A6E0BAF80800A0F50072013A0ED0B0F594
:1087E000007F0DD01120CDE90010E31C5B4A611C15
:1087F000601CF8F783F8FAF759FE91E02220F2E7BF
:108800001120F0E7BAF8020001280BD06770E7707A
:10881000277167712770BAF8222000214F48F9F7B5
:10882000C5FE7DE0BAF80800B0F5407F1AD0A0F58B
:108830004072013A14D0A0F54072023A14D0A0F56B
:108840004072033A12D01120CDE90010E31C00223F
:108850004249601CF8F752F8FAF728FE60E007E09A
:108860001220F1E71120EFE71120EDE72120EBE7DF
:10887000AB4501D027706770012D02D0022D1FD0AB
:108880002AE0BAF80C00012807D02770BAF8222095
:1088900000213248F9F78AFE1EE0BAF81000A0F570
:1088A0008071013908D0B0F5807F07D011230021F5
:1088B0002A48F8F7BBFD0FE02223F8E71123F6E77B
:1088C000BAF80C00012811D027706770BAF822207E
:1088D0002249601CF9F76AFE0298484502D0E77009
:1088E00027716771B9F1010F13D019E0BAF81000C0
:1088F000A0F50071013908D0B0F5007F07D0112331
:108900001649601CF8F792FDE6E72223F8E71123E9
:10891000F6E7BAF8140001281BD0E77027716771D9
:108920000396AB46CDF8089020680090A188ADF87A
:1089300004100199FAF7E8FB08F10108B8F1C80F33
:1089400003D3FEF713F84FF000080A2001F0E0F916
:10895000EEE6E01CF8F7FCFDE2E7000077000020FF
:1089600098AA00202DE9F04105460024A0460026E3
:10897000FBF750FA2D482E4F05E029190144097ADA
:108980003955641CE4B2082CF7D32844017C3972B1
:10899000017D427C41EA0261827CC37C120442EA8E
:1089A00003221143F960017E427D41EA0261827D2A
:1089B000C07D120442EA00200143796108221D496A
:1089C0001B4800F083F968B9FEF724F8397A884229
:1089D00008D2F86830B10021404600F0CDF80146D9
:1089E000012604E00121404600F0C6F801460020BF
:1089F00038610C2002F054FB1420FBF785FA002E9E
:108A000011D00D4DFDF738FF002405EB8420FDF754
:108A1000D3FE641CE4B21A2CF7D3FDF7B9FEBDE80F
:108A2000F041FEF7A7BDBDE8F0810000080200207C
:108A3000F0010020420000200098000810B500243A
:108A4000FDF7E8FF0146204600F096F80146BDE834
:108A500010400B2002F024BB2DE9F04105460E46E4
:108A60000024114F1CE0002204213846FEF700F8D4
:108A7000280605D4002210213846FDF7F9FF04E04E
:108A8000012210213846FDF7F3FFF9F701F8012222
:108A900004213846FDF7ECFF6806050E641CE4B2BD
:108AA000B442E0D3BDE8F081000C01402DE9F04173
:108AB00005460E460024114F15E0002204213846D9
:108AC000FDF7D6FFE80712D0012210213846FDF746
:108AD000CFFFF8F7DDFF012204213846FDF7C8FF7C
:108AE0006D08641CE4B2B442E7D3BDE8F081002213
:108AF00010213846FDF7BCFFEBE70000000C0140F9
:108B000070B505460C4C002208212046FDF7B0FF49
:108B100003218020FFF7A0FF08212846FFF79CFFD4
:108B200001210020FFF798FF2046BDE87040012298
:108B30000821FDF79DBF0000000C01400648018898
:108B4000491C018001884FF6F072914201D9012140
:108B500001800088704700004000002070B5044686
:108B600015460448204408302A46FEF716FE6019D0
:108B700080B270BD91020020024A02441172401C72
:108B800080B27047910200207CB500F077FF002290
:108B90008C21072001F0DCFB304C206200228C216C
:108BA000072001F0D5FB606203220021012001F0C3
:108BB000CFFBA062022104F10C00CDE900100D02F0
:108BC00000232A4626A1294801F0A0FE201D0321EA
:108BD000CDE9001000236A1025A1284801F096FE77
:108BE00004F108000421CDE9001000232A4624A145
:108BF000264801F08BFE04F110000521CDE900109C
:108C000000232A4622A1254801F080FE04F1140029
:108C10001021CDE9001000232A4621A1234801F0AC
:108C200075FE04F118000821CDE9001000232A4642
:108C30001FA1244801F06AFE04F11C00CDE9005098
:108C4000002312221AA1204801F060FE206801F0E2
:108C5000F1F8BDE87C4000F04DBF000000000020AE
:108C60007A69676265655F7461736B00B9AF00080C
:108C70006C65645F7461736B00000000ED70000848
:108C80006C63645F7461736B00000000616D0008C9
:108C90006B65795F7461736B00000000516D0008B3
:108CA0006D625F7274755F7461736B00FD730008B1
:108CB0006D625F7274755F6465616C5F7461736B24
:108CC0000000000075730008FD86000830B5002321
:108CD0000DE0C45CCD5CAC4202D24FF0FF3030BD41
:108CE00002D94FF0010030BD03F10103DBB2934222
:108CF000EFD3002030BD000000212648026842F07A
:108D0000010202604FF4A063491C026802F00202F3
:108D10000AB99942F8D10168890700D4FEE7C16910
:108D200041F08051C1611C490A6842F440420A6026
:108D30004268426042684260426842F48062426037
:108D40004268164B1A4042604268154B1A43426013
:108D5000026842F08072026002689201FCD50A68E3
:108D600042F480320A604A68D203FCD50A6842F4B1
:108D700000320A604A689203FCD5416821F0030181
:108D80004160416841F00201416041680907FCD53A
:108D9000704700000010024000700040FFFFC3B7A2
:108DA00000003408FFF7A8BF4FF0E021042804D0EA
:108DB000086920F0040008617047086940F0040069
:108DC0000861704730B587B040F20B60FFF76CFC6C
:108DD00040F20260FFF768FC4FF4C060FFF764FCEC
:108DE0004FF48073032218212048FDF747FE204DE1
:108DF000284600F03BFB7720ADF80C000024ADF8CE
:108E00000E40ADF8104040F2E7310591ADF8124048
:108E10008DF8184003A9284600F0A0FBADF80440E7
:108E20000120ADF800006A460021284600F0CCF988
:108E30001048808D08B1002200E01E220021284643
:108E400000F0D8FA60220021284600F0A9FA00229A
:108E50001146284600F0DEFA0121284600F0CFFB3B
:108E6000284600F076FB07B030BD00000008014046
:108E7000002C014098AA002030B587B040F2017064
:108E8000FFF712FC40F20260FFF70EFC40F20360B5
:108E9000FFF70AFC4FF4C060FFF706FC80230322B3
:108EA00018213E48FDF7EAFD3D4C0123032218211D
:108EB0002046FDF7E3FD0223032218212046FDF79B
:108EC000DDFD384D284600F0D1FA7720ADF80C00D2
:108ED0000024ADF80E40ADF8104040F2E7310591A6
:108EE000ADF812408DF8184003A9284600F036FB73
:108EF000ADF804400120ADF800006A460121284683
:108F000000F062F96A460221284600F05DF96A46DF
:108F10000321284600F058F9234CA08D08B1002207
:108F200000E01E220121284600F064FA602201219F
:108F3000284600F035FA00220121284600F06AFA9E
:108F4000A18D09B1002200E01E220221284600F076
:108F500051FA60220221284600F022FA0022022162
:108F6000284600F057FAA18D09B1002200E01E2228
:108F70000321284600F03EFA60220321284600F033
:108F80000FFA00220321284600F044FA284600F098
:108F900015F9284600F0DDFA07B030BD00080140A1
:108FA000000C01400004004098AA002030B587B0B2
:108FB00040F20370FFF778FB40F20260FFF774FBAA
:108FC0004FF4C060FFF770FB0123032218211E48F5
:108FD000FDF754FD1D4D284600F048FA7720ADF806
:108FE0000C000024ADF80E40ADF8104040F2E7311F
:108FF0000591ADF812408DF8184003A9284600F0FD
:10900000ADFAADF804400120ADF800006A46002139
:10901000284600F0D9F84FF496720021284600F057
:10902000E9F960220021284600F0BAF90022114631
:10903000284600F0EFF9284600F0C0F8284600F076
:1090400088FA07B030BD000000080140000C004065
:1090500030B587B040F20D60FFF726FB40F20460A8
:10906000FFF722FB4FF4C060FFF71EFB504C40237C
:10907000032218212046FDF701FD80230322182139
:109080002046FDF7FBFCA315032218212046FDF71F
:10909000F5FC6315032218212046FDF7EFFC454D32
:1090A000284600F0E3F97720ADF80C000024ADF875
:1090B0000E40ADF8104040F2E7310591ADF8124096
:1090C0008DF8184003A9284600F048FAADF804408E
:1090D0000120ADF800006A460021284600F074F82F
:1090E0006A460121284600F06FF86A4602212846A8
:1090F00000F06AF86A460321284600F065F82E4C15
:10910000A08D08B1002200E01E220021284600F0B8
:1091100071F960220021284600F042F90022114630
:10912000284600F077F9A18D09B1002200E01E2247
:109130000121284600F05EF960220121284600F056
:109140002FF900220121284600F064F9A18D09B110
:10915000002200E01E220221284600F04BF9602286
:109160000221284600F01CF900220221284600F0C6
:1091700051F9A18D09B1002200E01E2203212846E9
:1091800000F038F960220321284600F009F9002296
:109190000321284600F03EF90121284600F02FFA6D
:1091A000284600F00BF8284600F0D3F907B030BD90
:1091B000001001400034014098AA0020016841F0ED
:1091C000800101607047000030B5734B734C00297B
:1091D00029D0012960D002297ED0032922D1016A39
:1091E00021F480510162C16921F44071C161016AB9
:1091F000158841EA05310162016A21F400510162DA
:10920000016A958841EA05310162984201D0A04285
:1092100008D1416821F4804141604168128941EAE6
:109220008211416030BD016A21F001010162816952
:1092300021F003018161016A158829430162016AF5
:1092400021F002010162016A958829430162984276
:1092500001D0A042E6D1016A21F004010162016A55
:10926000538819430162016A21F008010162016A11
:10927000D38819430162416821F4807141604168DB
:10928000138919434160416821F4007141604168CC
:1092900052891143416030BD016A21F01001016221
:1092A000816921F440718161016A158841EA0511E3
:1092B0000162016A21F020010162016A958841EA98
:1092C00005110162984201D0A042E4D1016A21F067
:1092D00040010162016A00E01FE0538841EA031186
:1092E0000162016A21F080010162016AD38841EACA
:1092F00003110162416821F4806141604168138972
:1093000041EA83014160416821F4006141604168A4
:10931000528941EA8201416030BD016A21F48071C5
:109320000162C16921F00301C161016A158841EA46
:1093300005210162016A21F400710162016A9588C8
:1093400041EA05210162984201D0A042E4D1016ABC
:1093500021F480610162016A538841EA03210162BC
:10936000016A21F400610162016AD38841EA0321A4
:109370000162416821F4805141604168138941EAEA
:1093800003114160416821F40051416041685289F4
:1093900041EA0211416030BD002C0140003401401F
:1093A00000290ED0012914D002291BD0032907D18E
:1093B000C16921F4E041C161C16941EA0221C16191
:1093C0007047816921F07001816181691143816178
:1093D0007047816921F4E0418161816941EA02219C
:1093E00081617047C16921F07001C161C169114398
:1093F000C1617047002907D0012907D0022907D091
:10940000032900D10264704742637047826370474A
:10941000C263704700290ED0012914D002291BD045
:10942000032907D1C16921F40061C161C16941EA21
:109430000221C1617047816921F008018161816960
:10944000114381617047816921F400618161816903
:1094500041EA022181617047C16921F00801C161BF
:10946000C1691143C16170474162704710B5344A08
:10947000811A141590424DD014DCB0F1804F2DD0DC
:109480003049401832D0A0423AD0B0F5006F55D1E3
:1094900040F203442046FFF723F92046BDE8104080
:1094A000FFF710B9A1423FD0B1F58E3F0CD0B1F516
:1094B000923F43D140F20D342046FFF711F9204688
:1094C000BDE81040FFF7FEB840F20B342046FFF72E
:1094D00007F92046BDE81040FFF7F4B82046FFF733
:1094E000FFF82046BDE81040FFF7ECB840F2014419
:1094F0002046FFF7F5F82046BDE81040FFF7E2B838
:1095000040F202442046FFF7EBF82046BDE8104049
:10951000FFF7D8B840F204442046FFF7E1F82046B0
:10952000BDE81040FFF7CEB840F205442046FFF7F3
:10953000D7F82046BDE81040FFF7C4B810BD0000C2
:109540000010004000FCFFBF016821F00101016034
:109550007047016841F001010160704730B50A8829
:1095600082621C4B1C4A98420DD0B0F1804F0AD049
:109570001A4CA04207D01A4CA04204D0194CA04269
:1095800001D090420BD1046824F070040460046898
:109590004D882C43046004688D882C4304608C68DB
:1095A000C462114CA0420AD0104CA04207D00468FB
:1095B00024F4407404600468CD882C43046098420D
:1095C00001D0904201D1097B0163416941F0010161
:1095D000416130BD002C01400034014000040040D6
:1095E00000080040000C0040001000400014004043
:1095F000C2680A43C2607047C943016170470129CC
:1096000004D0416C21F4004141647047416C41F445
:1096100000414164704700210180418081804FF604
:10962000FF728260C18001737047000010B50C4961
:109630000C4B0A681968541A012C0FD0914203D9B7
:109640008A1AB2F5847F09D8074A914202D3A2F25E
:1096500009111960196801F8010B196010BD0000AB
:10966000500000204C0000202304002070B5044668
:109670000D460020174BE21A1E159C4216D008DC3E
:10968000154962180ED0B24217D10220FEF78EFFA4
:1096900013E0B2420ED0B2F56C4F0ED10320FEF7AC
:1096A00085FF0AE00220FEF781FF06E00220FEF7B8
:1096B0007DFF02E00220FEF779FF00EB5500B0FBD2
:1096C000F5F04FF6F071014000F00F021143A16078
:1096D00070BD0000004C004000BCFFBF10B54FF44F
:1096E000A060FEF7D7F8002202212520FEF784F8BB
:1096F00040F20E60FEF7D8FF134C204600F02EF823
:109700004FF4E1312046FFF7B1FF0021204600F081
:10971000EDF80021204600F0D7F80021204600F0A7
:10972000C1F80421204600F0C5F80821204600F0C9
:10973000D3F8204600F05AF82046BDE8104040F229
:10974000053100F083B80000003801404068C0F3E4
:1097500008007047C1F308014160704710B5214A05
:10976000811A1315904228D00EDC1F4940181AD0D8
:10977000984236D140F212442046FEF7B1FF20460F
:10978000BDE81040FEF79EBF994220D0B1F56C4F66
:1097900027D140F20E342046FEF7A2FF2046BDE856
:1097A0001040FEF78FBF40F211442046FEF798FFAD
:1097B0002046BDE81040FEF785BF40F21344204626
:1097C000FEF78EFF2046BDE81040FEF77BBF40F25B
:1097D00014442046FEF784FF2046BDE81040FEF703
:1097E00071BF10BD004C004000BCFFBFC16841F418
:1097F0000051C160704700EB9110006801F01F023A
:1098000001219140084201D001207047002070479B
:10981000426922F400724261426901F400710A4314
:1098200042617047426922F480724261426901F4E8
:1098300080710A434261704700EB9110026801F0A9
:109840001F03012199408A430260704700EB911089
:10985000026801F01F03012199400A43026070472A
:10986000C1F3044301229A4000EB9150D2430260BD
:10987000704730B5C1F38912825801F01F040125E9
:1098800005FA04F31A4000EB91500068C1F304415B
:1098900005FA01F31840002802D00AB1012030BDBA
:1098A000002030BDC26822F4C062C260C2680A43B0
:1098B000C2607047C26822F00402C260C26801F050
:1098C00004010A43C2607047026922F440520261F7
:1098D00002690A4302617047C26822F00802C2604E
:1098E000C26801F008010A43C2607047C26822F4EE
:1098F0008052C260C2680A43C26070472DE9F05FBF
:10990000F8F7E6F80024144E144F154D4FF00108F7
:109910004FF064094FF0FA0A4FF4FA7B05EB44105C
:10992000047746608760417F21F001014177A0F80C
:109930001480A0F81690A0F818A0A0F81AB0012C76
:1099400001D0062C01D19621C182FCF75DFE641C7A
:10995000082CE3DBBDE8F09F0D3E0008093B000842
:109960004C0600200169D0E901329A60D0E9012358
:109970005A604A68824201D182684A6000220261CC
:109980000868401E0860704700F1080141604FF010
:10999000FF328260C16001610021016070470021D7
:1099A0000161704730B50C68621C02D000F10802FA
:1099B00002E0026904E01A4653681D68A542FAD91C
:1099C00053684B6099608A60516008610168491C66
:1099D000016030BD42684A6093688B60936859604B
:1099E000916008610168491C0160704770B50D46BF
:1099F000104A4FF4804144F62064002807D000202C
:109A0000401CA042FCD31046FDF72EF806E010469D
:109A1000FDF72CF80020401CA042FCD3064840F281
:109A200007311DB1BDE87040FFF710BFBDE87040C1
:109A3000FFF702BF001001400044004010B54FF096
:109A4000804400212046FFF70FFD01212046FFF74B
:109A5000D3FD2046BDE81040FFF776BD10B54FF0AE
:109A6000804400212046FFF7FFFC01212046FFF73C
:109A7000C3FD2046BDE81040FFF76BBD502080F3CA
:109A80001188BFF34F8FBFF36F8F09494868401C9F
:109A9000486001280AD10748006810F0FF0F05D080
:109AA00040F2B91204A10FA0F9F7ACBE7047000054
:109AB0005801002004ED00E02E2E5C4672656552D0
:109AC000544F535C706F727461626C655C525644A3
:109AD000535C41524D5F434D34465C706F72742E3F
:109AE000630000004572726F723A25732C25640D75
:109AF0000A00000010B5094C6068002805D14FF439
:109B0000E07207A111A0F9F77DFE6068401E606059
:109B1000002801D180F3118810BD000058010020F9
:109B20002E2E5C4672656552544F535C706F727492
:109B300061626C655C525644535C41524D5F434DCB
:109B400034465C706F72742E630000004572726F51
:109B5000723A25732C25640D0A00000070B50028A8
:109B60002AD008380446154D6068E968084205D1D6
:109B70004FF4A07212A11CA0F9F744FE206828B18E
:109B800040F241120EA118A0F9F73CFE6068E968A6
:109B9000084211D02268002A0ED18843606000F08C
:109BA000C3FA60686968084468602046FEF720F9D7
:109BB000BDE8704001F0CAB870BD0000400100204F
:109BC0002E2E5C4672656552544F535C706F7274F2
:109BD00061626C655C4D656D4D616E675C68656169
:109BE000705F342E630000004572726F723A257305
:109BF0002C25640D0A00000006484FF47A710068B5
:109C0000B0FBF1F14FF0E020491E416107210161F5
:109C1000704700003000002010B5F6F7EDFA104C48
:109C200010280CD300F1E02090F8F003217888424E
:109C300005D24FF440720BA115A0F9F7E3FD1848C7
:109C40000068A16800F4E060884207D9BDE81040D0
:109C50004FF4447203A10EA0F9F7D4BD10BD00006B
:109C6000580100202E2E5C4672656552544F535C9D
:109C7000706F727461626C655C525644535C415201
:109C80004D5F434D34465C706F72742E630000006C
:109C90004572726F723A25732C25640D0A0000001C
:109CA0000CED00E010B50022064B53F832401CB119
:109CB000521C082AF9D310BD43F8321003EBC2013D
:109CC000486010BD4C07002070B504460D4616468E
:109CD000FFF7D4FE94F944304FF000005B1C01D133
:109CE00084F8440094F94510491C01D184F84500DA
:109CF000FFF700FFA06B28B93246294604F1240083
:109D000000F030F92046BDE87040FEF7BBBA000015
:109D100010B504460020002C10D00E48006B28B16E
:109D200040F2CF420CA111A0F9F76CFD00F0FCF954
:109D300000212046FDF74CFE01F008F8002807D16D
:109D40000E494FF080500860BFF34F8FBFF36F8F05
:109D500010BD0000F00000202E2E5C46726565529A
:109D6000544F535C7461736B732E63004572726F52
:109D7000723A25732C25640D0A00000004ED00E002
:109D80002DE9F04105460E460024002D05D140F294
:109D900079421DA121A0F9F735FD2EB940F27A4292
:109DA00019A11EA0F9F72EFD204F386B28B140F203
:109DB0007B4215A119A0F9F725FD00F0B5F9FA6865
:109DC0002B689919934205D98B4208D9914206D93B
:109DD000012404E08B4201D8914200D9012429607A
:109DE0001CB1881A0021FDF7F3FD00F0AFFF002839
:109DF00007D10F494FF080500860BFF34F8FBFF37A
:109E00006F8FBDE8F08100002E2E5C4672656552B2
:109E1000544F535C7461736B732E63004572726FA1
:109E2000723A25732C25640D0A000000F000002012
:109E300004ED00E070B50446FFF720FE234D04B9A1
:109E40002C68201DFFF78EFD58B9E06A204A00EB10
:109E5000800152F8211021B90121814028698843ED
:109E60002861A06A18B104F11800FFF77BFD686A49
:109E7000401C68622868844207D1211D1548FFF7FD
:109E8000A9FD6868401C686007E0A868401EA860DB
:109E90002046FDF7B8FEFEF749F9FFF72BFE68698B
:109EA000002812D0286884420FD1286B28B140F2D4
:109EB000654209A10DA0F9F7A5FC10494FF08050AB
:109EC0000860BFF34F8FBFF36F8F70BDF0000020AD
:109ED0008C070020480A00202E2E5C4672656552D1
:109EE000544F535C7461736B732E63004572726FD1
:109EF000723A25732C25640D0A00000004ED00E081
:109F000001490120C8617047F000002070B5044687
:109F10000D46002C05D140F6063208A10CA0F9F739
:109F200071FC0F48016820461831FFF73BFD2846B9
:109F3000BDE870400121FDF74BBD00002E2E5C46B0
:109F400072656552544F535C7461736B732E63007A
:109F50004572726F723A25732C25640D0A00000059
:109F6000F000002070B506460D461446002E05D1BF
:109F700040F6313209A10EA0F9F744FC10480168FF
:109F800030461831FFF726FD0CB14FF0FF35214662
:109F90002846BDE87040FDF71BBD00002E2E5C4634
:109FA00072656552544F535C7461736B732E63001A
:109FB0004572726F723A25732C25640D0A000000F9
:109FC000F000002070B50446002839D01D4DE06A2D
:109FD0002968C96A884233D2A069002804DB28684E
:109FE000C06AC0F12000A061E06A174E00EB80005B
:109FF000616906EB800081421FD1201DFFF7B2FC92
:10A00000012150B9E06A00EB800256F8222022B903
:10A010002A6901FA00F082432A612868C06AE06276
:10A020002A6981401143296100EB800006EB800022
:10A03000211DBDE87040FFF7CDBC2868C06AE06212
:10A0400070BD0000F00000208C07002010B5044611
:10A05000002C05D140F6C13204A109A0F9F7D2FBCA
:10A060000B48016A2160C068606010BD2E2E5C46FE
:10A0700072656552544F535C7461736B732E630049
:10A080004572726F723A25732C25640D0A00000028
:10A09000F00000201CB517480024CDE900402346FD
:10A0A000822215A1164800F031FC012801D100F0F0
:10A0B000C3FE01280AD0401C1BD102B040F28472BA
:10A0C000BDE810400FA114A0F9F79CBB502080F30D
:10A0D0001188BFF34F8FBFF36F8F06484FF0FF31EA
:10A0E0002C38816201214161C460BDE81C4000F050
:10A0F00091B81CBD1C01002049444C4500000000E3
:10A100008D7C00082E2E5C4672656552544F535C60
:10A110007461736B732E63004572726F723A2573AC
:10A120002C25640D0A0000000248016B491C0163E4
:10A1300070470000F000002070B5144D286B002817
:10A1400002D00120E86170BD0020E8612869B0FA02
:10A1500080F0C0F11F000E4E00EB800456F8240082
:10A1600028B940F6F6220BA10FA0F9F74BFB06EB3E
:10A17000840041684968416000F10802914201D1C0
:10A18000496841604068C068286070BDF0000020E8
:10A190008C0700202E2E5C4672656552544F535C2E
:10A1A0007461736B732E63004572726F723A25731C
:10A1B0002C25640D0A000000044805490068096860
:10A1C000884201D0012070470020704750000020D5
:10A1D0004C00002070B504460E460D4D00220821AB
:10A1E0002846FCF745FC0321A020FEF735FCA0061D
:10A1F000000E0621FEF730FC04213046FEF756FC27
:10A200002846BDE8704001220821FCF731BC00005F
:10A21000000C01401CB52F4C20682F49884205D105
:10A2200040F259122DA138A0F9F7ECFA20682A491A
:10A23000491E884205D14FF4AD7228A132A0F9F72A
:10A24000E1FA354C20780190FF20207020780090B2
:10A250009DF800009DF8001000F0F000884205D045
:10A2600040F273121DA128A0F9F7CCFA9DF8000066
:10A270002A4A00F0500010700720906006E09068B5
:10A28000401E90609DF80000400000909DF8000086
:10A290000006F4D4107A000200F4E06090600198A7
:10A2A00020700C482030016841F4700101600168A1
:10A2B00041F070410160FFF79FFC00205060F5F70E
:10A2C00063FF1748016841F040410160F5F74CFF1A
:10A2D00000201CBD00ED00E071C20F412E2E5C4637
:10A2E00072656552544F535C706F727461626C6535
:10A2F0005C525644535C41524D5F434D34465C7052
:10A300006F72742E630000004572726F723A25738B
:10A310002C25640D0A00000000E400E05801002034
:10A3200034EF00E010B5502080F31188BFF34F8F59
:10A33000BFF36F8F00F0A4FB18B104494FF08050B9
:10A340000860002080F3118810BD000004ED00E0DB
:10A35000F8B505460E461746002D05D14FF4C472D8
:10A360000BA110A0F9F74EFA86B105FB06F05430A8
:10A37000FEF778F804463CB104F154023B463146FE
:10A3800028460094FDF796FC2046F8BD0020EEE735
:10A390002E2E5C4672656552544F535C717565751F
:10A3A000652E63004572726F723A25732C25640D19
:10A3B0000A0000002DE9FF4F83B004468A469B4601
:10A3C0000026002C05D140F2DC4258A15CA0F9F730
:10A3D00019FABAF1000F07D1206C28B140F2DD4222
:10A3E00052A157A0F9F70EFA00F036FB38B90598DC
:10A3F00028B14FF49C624DA151A0F9F703FA4FF038
:10A4000000094FF08057DFF84881FFF737FBA56B55
:10A4100095B3E66851462046FDF7AAFBBBF1000F55
:10A4200013D0E660606A50B104F1240000F040FCF3
:10A4300028B1C8F80070BFF34F8FBFF36F8FFFF7DD
:10A4400059FB012007B0BDE8F08F6D1EA5632068A1
:10A4500010B9FEF78DF8606020690028EFD004F194
:10A46000100000F025FC0028E9D0C8F80070BFF308
:10A470004F8FBFF36F8FE2E7FFE7059808B126B172
:10A4800007E0FFF737FB0020DCE701A8FFF7DEFD60
:10A490000126FFF72FFBFFF747FEFFF7EFFA94F9CE
:10A4A0004400401C01D184F8449094F94500401CBC
:10A4B00001D184F84590FFF71DFB05A901A800F024
:10A4C000DDF958B12046FDF7DDFE00F03FFC2046E7
:10A4D000FDF7D8FC002898D00020B3E72046FDF710
:10A4E000D1FCE0B1206830B9FFF7C8FA6068FFF727
:10A4F00069FDFFF7FFFA04F124000599FFF706FD57
:10A500002046FDF7BFFE00F021FC00287FF47DAF60
:10A51000C8F80070BFF34F8FBFF36F8F75E7204609
:10A52000FDF7B0FE00F012FC6FE700002E2E5C4637
:10A5300072656552544F535C71756575652E630085
:10A540004572726F723A25732C25640D0A00000063
:10A5500004ED00E070B504460D46002C05D140F234
:10A560001B121DA121A0F9F74DF9FFF787FAD4E9D5
:10A570000F20216802FB001161600021A1632168A6
:10A58000A160E06B2268216C401E00FB0121E160AC
:10A590004FF0FF3084F8440084F8450004F11000C7
:10A5A0004DB1FFF7F1F904F12400FFF7EDF9FFF7E2
:10A5B000A1FA012070BD21690029F8D000F078FBD4
:10A5C0000028F4D00D494FF080500860BFF34F8F42
:10A5D000BFF36F8FEBE700002E2E5C46726565526D
:10A5E000544F535C71756575652E63004572726FCB
:10A5F000723A25732C25640D0A00000004ED00E07A
:10A600002DE9FF4782B004468A4698460025002C73
:10A6100005D140F2D92254A158A0F9F7F3F8BAF1C4
:10A62000000F07D1206C28B140F2DA224EA153A0CE
:10A63000F9F7E8F8B8F1020F08D1E06B012805D06E
:10A6400040F2DB2248A14DA0F9F7DCF800F004FA53
:10A6500038B9049828B140F2DE2243A147A0F9F7A7
:10A66000D1F84FF000094FF08056484FFFF706FA37
:10A67000A06BE16B884206D3B8F1020F03D00498B7
:10A6800060B37DB333E0424651462046FDF784FA7D
:10A69000A16C51B141462046FDF710FCC0B13E60AF
:10A6A000BFF34F8FBFF36F8F12E0616A51B104F1B6
:10A6B000240000F0FDFA58B13E60BFF34F8FBFF3A6
:10A6C0006F8F05E020B13E60BFF34F8FBFF36F8FF8
:10A6D000FFF710FA012006B0BDE8F087FFF70AFA8D
:10A6E0000020F8E7FFE76846FFF7B0FC0125FFF719
:10A6F00001FAFFF719FDFFF7C1F994F94400401C76
:10A7000001D184F8449094F94500401C01D184F8AB
:10A710004590FFF7EFF904A9684600F0AFF830B1B3
:10A720002046FDF7AFFD00F011FB0020D3E72046E7
:10A73000FDF7B5FB88B104F110000499FFF7E6FBC3
:10A740002046FDF79FFD00F001FB00288ED13E6002
:10A75000BFF34F8FBFF36F8F88E72046FDF792FD61
:10A7600000F0F4FA82E700002E2E5C467265655216
:10A77000544F535C71756575652E63004572726F39
:10A78000723A25732C25640D0A00000004ED00E0E8
:10A790002DE9F0470446894615469846002C05D118
:10A7A00040F29F322CA131A0F9F72CF8B9F1000F3B
:10A7B00007D1206C28B14FF4687227A12BA0F9F7BC
:10A7C00021F8B8F1020F08D1E06B012805D040F262
:10A7D000A13221A125A0F9F715F8FFF71DFA5020A5
:10A7E000EFF3118780F31188BFF34F8FBFF36F8FA3
:10A7F000A06BE16B884207D3B8F1020F04D00020B0
:10A8000087F31188BDE8F08794F9456042464946D0
:10A810002046FDF7C1F9701C04D0761C84F8456011
:10A820000120EDE7A06C012648B141462046FDF726
:10A8300045FB0028F4D0002DF2D02E60F0E7606ACE
:10A840000028EDD004F1240000F032FA0028E7D00F
:10A85000002DE5D02E60E3E72E2E5C467265655232
:10A86000544F535C71756575652E63004572726F48
:10A87000723A25732C25640D0A00000070B5044659
:10A880000D46002C05D140F6CB3216A11AA0F8F7E0
:10A89000B9FF2DB940F6CC3212A117A0F8F7B2FFDC
:10A8A000FFF7ECF8184AD06829684B1C08D02368D9
:10A8B000126A934206D06268824203D801240DE0F6
:10A8C00000240BE06268801A884206D2081A2860C9
:10A8D0002046FFF7BBFB002400E00124FFF70AF944
:10A8E000204670BD2E2E5C4672656552544F535CF7
:10A8F0007461736B732E63004572726F723A2573C5
:10A900002C25640D0A000000F00000202DE9FF5FF7
:10A910008146DDE90E788A4616469B46B000FDF773
:10A92000A1FD054628000AD05C20FDF79BFD0446EA
:10A930000CB1256304E02846FFF710F900E000247D
:10A940008CB10020CDE90240CDE900785B4632466B
:10A9500051464846FDF7C2F92046FDF771F801203F
:10A9600004B0BDE8F09F4FF0FF30F9E72DE9F0416A
:10A9700004460D4690461F460126002C05D141F2A3
:10A98000FD0229A12DA0F8F73DFFFFF777F80FB1E1
:10A99000606D386094F85800022184F85810B8F1BE
:10A9A000050F13D2DFE808F01203070B0D00616DED
:10A9B000294361650AE0616D491C616506E06565D2
:10A9C00004E0022801D0656500E00026012826D1B8
:10A9D000201DFEF7C7FF1D4DE06A01212A69814055
:10A9E000114329611A4900EB800001EB8000211D11
:10A9F000FEF7F0FFA06A28B141F235120AA10FA0BC
:10AA0000F8F700FFE06A2968C96A884207D9114946
:10AA10004FF080500860BFF34F8FBFF36F8FFFF789
:10AA200069F83046BDE8F0812E2E5C4672656552AD
:10AA3000544F535C7461736B732E63004572726F75
:10AA4000723A25732C25640D0A000000F0000020E6
:10AA50008C07002004ED00E005484169002903D07F
:10AA6000006B18B10020704701207047022070472A
:10AA7000F00000200148C06870470000F00000208E
:10AA80002DE9F04100262E4F386B002808D0B86918
:10AA9000401CB861F86900B101263046BDE8F0817C
:10AAA000FD686D1CFD608DB9786B006828B140F6BB
:10AAB000D91224A128A0F8F7A5FE786BB96B7963A9
:10AAC000B863386A401C3862FDF730FBB86ADFF8BB
:10AAD000988085420DD3786B006838B1786BC06878
:10AAE000C468606885420ED2B86202E04FF0FF3061
:10AAF000B8623868C06A00EB800058F8200001286E
:10AB0000C8D90126C6E7201DFEF72CFFA06A18B1A0
:10AB100004F11800FEF726FFE06A01213A6981403E
:10AB20001143396100EB800008EB8000211DFEF726
:10AB300051FFE06A3968C96A8842CCD30126CAE766
:10AB4000F00000202E2E5C4672656552544F535C17
:10AB50007461736B732E63004572726F723A257362
:10AB60002C25640D0A0000008C0700202DE9F04719
:10AB700081460F4616469846FEF780FF1D4D286811
:10AB800090F85800022817D02C68606D20EA090060
:10AB900060652968012081F85800B8F1000F0BD0DA
:10ABA00001214046FCF714FF13494FF08050086024
:10ABB000BFF34F8FBFF36F8FFEF79CFFFEF75EFF73
:10ABC00016B12868406D3060286890F85800012858
:10ABD0000DD02868416DB9434165012429680020E2
:10ABE00081F85800FEF786FF2046BDE8F087002474
:10ABF000F4E70000F000002004ED00E070B504462A
:10AC0000002600283CD01F4D2868844205D040F61D
:10AC1000C7621DA121A0F8F7F5FD206D28B940F607
:10AC2000C96219A11DA0F8F7EDFD206D401E206539
:10AC3000E26CE16A914223D010BB201DFEF792FE28
:10AC40001A4A012150B9E06A00EB800352F8233020
:10AC500023B92B6901FA00F083432B61E06CE062B9
:10AC6000C0F12000A061E06A2B698140194329618D
:10AC700000EB800002EB8000211DFEF7ABFE0126F9
:10AC8000304670BDF00000202E2E5C467265655285
:10AC9000544F535C7461736B732E63004572726F13
:10ACA000723A25732C25640D0A0000008C070020E1
:10ACB0002DE9F041C068C468002C05D140F661322E
:10ACC00016A11BA0F8F79EFD04F118000746FEF739
:10ACD00049FE1B4D2A6B012662B139461948FEF721
:10ACE00079FEE06A2968C96A884215D90120EE61B7
:10ACF000BDE8F081201DFEF735FEE06A2A6906FAFC
:10AD000000F111432961104900EB800001EB800044
:10AD1000211DFEF75FFEE4E70020E9E72E2E5C46EA
:10AD200072656552544F535C7461736B732E63008C
:10AD30004572726F723A25732C25640D0A0000006B
:10AD4000F0000020340A00208C0700202DE9F0419B
:10AD5000002400272B4D286B002805D14FF4FD62FD
:10AD600029A12EA0F8F74EFDFEF788FE286B401EA5
:10AD70002863286BF0BBA868E0B3DFF8B080012639
:10AD80001DE0D8F80C00C46804F11800FEF7EAFDD5
:10AD9000201DFEF7E7FDE06A2A6906FA00F111437B
:10ADA0002961234900EB800001EB8000211DFEF7A3
:10ADB00011FEE06A2968C96A884200D3EE61D8F8BA
:10ADC00000000028DDD10CB1FDF7B0F9AC6944B149
:10ADD000FFF756FE00B1EE61641E002CF8D1002092
:10ADE000A861E86930B10127124938070860BFF34C
:10ADF0004F8F00E001E0BFF36F8FFEF77BFE384618
:10AE0000BDE8F081F00000202E2E5C467265655290
:10AE1000544F535C7461736B732E63004572726F91
:10AE2000723A25732C25640D0A000000340A0020B4
:10AE30008C07002004ED00E01CB50024FCF746FE62
:10AE40000C48006860B10B481F21001DCDE90010BF
:10AE500000234FF4827208A10948FFF757FD04460A
:10AE60002CB940F2331207A10CA0F8F7CBFC204616
:10AE70001CBD00002C010020546D7220537663002D
:10AE8000718200082E2E5C4672656552544F535CE9
:10AE900074696D6572732E63000000004572726FF5
:10AEA000723A25732C25640D0A0000002DE9FF4736
:10AEB000DDF830A005460E46904699460027002D45
:10AEC00005D14FF4D37215A11AA0F8F79BFC1D4CC5
:10AED0002068F8B10096CDF804800295062E13DAAA
:10AEE000FFF7BAFD022807D000231A4669462068FA
:10AEF000FFF786FB07460DE00023524669462068AF
:10AF0000FFF77EFB074605E000234A466946FFF748
:10AF10003FFC074604B03846BDE8F0872E2E5C465D
:10AF200072656552544F535C74696D6572732E631C
:10AF3000000000004572726F723A25732C25640D73
:10AF40000A0000002C0100202DE9F041044627787A
:10AF50006578A0780002E178084486B23846FBF7AD
:10AF60006DFD084901EB40004078A84202D0002066
:10AF7000BDE8F0813246211D3846BDE8F041FAF7C0
:10AF8000C7B8000030B1000810B500200121FDF75E
:10AF9000F3FD0146BDE81040002000F081B800003C
:10AFA0000349024808600349086070471A030020FB
:10AFB0004C0000205000002000F004F80520FEF7AF
:10AFC000A7FEF9E72DE9F04100242F4E2F4F06E0B0
:10AFD000F7F7C4FF02463888411C3980325438885C
:10AFE000892803D2FFF7E8F80028F1D1388809282A
:10AFF00048D330E0305D552802D0641CA4B22AE06A
:10B0000030194278AA2A02D0641CA4B223E08278C4
:10B01000022A02D0A41CA4B21DE082791202C379D4
:10B0200009321A4495B2892D02D9E41CA4B212E067
:10B03000A94214DB691E89B2FBF7DEFC2544A9197D
:10B0400011F8011C884202D0E41CA4B203E020469F
:10B05000F8F7F4FEACB23888011B0929CADA38883F
:10B06000001B80B2388000280CD024B9892802D374
:10B070000124401E388031193A88BDE8F041024869
:10B08000FCF78BBBBDE8F0810802002034000020F3
:10B09000002804D0002902D0491E89B2FCD2704792
:10B0A00070B506460D46114C55202070AA206070E0
:10B0B0000220A070FDF742FD0021E1702071667151
:10B0C000280AA071E5710935ADB2681E81B220462B
:10B0D000FBF792FC611901F8010C2046FCF780FB9C
:10B0E00081B22046BDE87040FFF7D2BF9102002038
:10B0F00010B5044600210220FFF7D2FF002C12D029
:10B100000020012C0DD0022C0DD1074981F85100EF
:10B110004FF47A704865C821BDE810401920FBF74C
:10B12000A9BF0249086010BD7405002080000020FE
:10B13000010102040304100218021C0465046602E3
:10B140006701680169040000FF00000000C1814040
:10B1500001C0804101C0804100C1814001C08041E7
:10B1600000C1814000C1814001C0804101C08041D7
:10B1700000C1814000C1814001C0804100C18140C7
:10B1800001C0804101C0804100C1814001C08041B7
:10B1900000C1814000C1814001C0804100C18140A7
:10B1A00001C0804101C0804100C1814000C1814097
:10B1B00001C0804101C0804100C1814001C0804187
:10B1C00000C1814000C1814001C0804101C0804177
:10B1D00000C1814000C1814001C0804100C1814067
:10B1E00001C0804101C0804100C1814000C1814057
:10B1F00001C0804101C0804100C1814001C0804147
:10B2000000C1814000C1814001C0804100C1814036
:10B2100001C0804101C0804100C1814001C0804126
:10B2200000C1814000C1814001C0804101C0804116
:10B2300000C1814000C1814001C0804100C1814006
:10B2400001C0804101C0804100C1814000C0C101F6
:10B25000C30302C2C60607C705C5C404CC0C0DCD86
:10B260000FCFCE0E0ACACB0BC90908C8D81819D9F6
:10B270001BDBDA1A1EDEDF1FDD1D1CDC14D4D51526
:10B28000D71716D6D21213D311D1D010F03031F116
:10B2900033F3F23236F6F737F53534F43CFCFD3D46
:10B2A000FF3F3EFEFA3A3BFB39F9F83828E8E92936
:10B2B000EB2B2AEAEE2E2FEF2DEDEC2CE42425E5E6
:10B2C00027E7E62622E2E323E12120E0A06061A156
:10B2D00063A3A26266A6A767A56564A46CACAD6D06
:10B2E000AF6F6EAEAA6A6BAB69A9A86878B8B97976
:10B2F000BB7B7ABABE7E7FBF7DBDBC7CB47475B5A6
:10B3000077B7B67672B2B373B17170B05090915195
:10B310009353529296565797559594549C5C5D9DC5
:10B320005F9F9E5E5A9A9B5B9959589888484989B5
:10B330004B8B8A4A4E8E8F4F8D4D4C8C4484854565
:10B34000874746868242438341818040E001C003B3
:10B35000A0058007000FE01500000000E001C00319
:10B36000A0058007000FE015000000008CB3000866
:10B3700000000020B80100003C070008B0B300083E
:10B38000B801002048AD0000343800080132045AEA
:10B390000E27070BC60102030405060708090A0564
:10B3A0001FAAAAAAAA33C8414370420231C00000B2
:0400000508000131BD
:00000001FF
